:020000041100E9
:10300000002373B52B4D2C4C28006361022601F080
:1030100069F94021FE2221742800284B009601F016
:10302000B3F9002836D1217CFF222800244B0096DA
:1030300001F0AAF900282DD1224BA2899A4226D16B
:10304000E389214A93420DD1204B6361204B2268D2
:10305000002A03D1002B01D043CB43C4280001F048
:103060007FF973BD1B4A934201D00023EFE71A4B4F
:103070001A4A1B68934206D9C02304222800217CE7
:103080009B0001F0F7F9114B6361154BDFE700235B
:103090002374EAE7CC233821AC2228009B01217459
:1030A00001F0E8F90028F2D10E4B63610E4BE38189
:1030B0000E4BCCE7643CFF1F105CFF1F1C5CFF1F26
:1030C0001E5CFF1F595900008305000011410011CB
:1030D000F0BC001182150000345CFF1F8713000054
:1030E000FCBC0011C9410011AAAAFFFFE4BC0011F9
:1030F000F7B5164B0192C318021D002000938823D8
:103100005B05D3181B685C1C1AD09CB2402C18D8E5
:103110008D781E0CAC466746CD782D023D43AE42FD
:1031200006D1019800280ED110000C70240A4C70B2
:1031300003249BB20733A343D218009B9A42DED3E9
:10314000FEBD4432F9E71000FAE7C046FC0F00006C
:10315000802213B503000324019189B25201073183
:103160009B18A14304305A1A88235B05C3181B68B7
:10317000591C03D190429241104016BD99B240298A
:1031800007D80B000733A343C0189042ECD30020AC
:10319000F3E74430F9E7134B134A1B68126810B584
:1031A000FA24934201D81A00F824104BE4021B6859
:1031B0009A4210D813000E4A12689A420ED3013375
:1031C00007D1F823DB029C4203D10A49054808F0E5
:1031D00003FD200010BDFC24E402ECE7FE24E40221
:1031E000F7E7C04600C0071100D0071100E0071143
:1031F00000F00711FFFFFF7FF0B59BB015000490B2
:103200000391402A00D9A0E006AB59801A80FFF74D
:10321000C2FF0400042816D9002206A9FFF768FFA0
:10322000052810D906AB1B88AB420CD1002D07D066
:10323000514B2A000499C01808F0CEFB002802D197
:1032400001201BB0F0BD06AB1D8020000699FFF7E2
:103250007FFF041E7BD1069B0793FFF79CFF802313
:103260005B01C618802307001B039E4201D3F8268A
:10327000F60288235B05F31801931B68013302D023
:10328000019808F0B1FA3D49019808F0A5FC3B1DF2
:103290000293331D05938822029B52059B181B68DD
:1032A00008935A1C3CD044219AB20091402A04D879
:1032B0000320D11D814389B2009103991B0C8B42DD
:1032C00024D0402A22D80122300008A9FFF710FF9D
:1032D000021E1BD1380008A9FFF70AFF04000428CA
:1032E00031D9009A059B9B1880225201B218934253
:1032F00040D288235B05C118009A09A808F0CCFBCE
:103300001D4B009A09A9F01808F046FC009A029B90
:103310009446634402931A4B029AFB189A42BAD31A
:1033200088235B05FC1821680198013908F054FCDA
:10333000200008F059FA039A07AB5A803000079929
:10334000FFF706FF0400002C03D1002079E70428D2
:10335000FBD988235B05E018069908F03DFC0323A0
:10336000EA1C9A4300D16BE7034B0499E01808F07C
:1033700013FC65E70424ECE704000011FFFFFF7F66
:10338000F80F0000F7B505001400402A21D80027E7
:1033900001AE71803780FFF7FEFE042816D93A008F
:1033A0003100FFF7A5FE042810D93688BC420BD0A7
:1033B000BD4209D0221CB44200D9321C064B92B245
:1033C000C118280008F068FB30B2FEBDC04300B24F
:1033D000FBE703204042F8E70400001137B5042260
:1033E00004000D0001A81649FFF7CCFF02000428D5
:1033F0000BD1019BA34208D3AB4204D0104901A8D2
:103400000195FFF7F9FE01203EBD0E4C2368200018
:10341000019308F0E9F9019920000139019108F0C0
:10342000DBFB80235B01E418074B9C42EED10422B6
:10343000034901A80195FFF7DFFE0020E4E7C0463D
:103440005555000000C007110000081130B589B0C3
:1034500008F002FA10226946254808F03DF9254B8C
:10346000009A9A420ED1019B029A0F2B33D8002169
:1034700001240698013B08D2002900D00292029B49
:10348000013331D10023029325E0551CF2D1020013
:103490002100EFE710341022200004A908F01CF9E5
:1034A000029B013301D1069B0293882304995B059B
:1034B000C918059B06981A03120B049105928142C4
:1034C00003D02B4201D108F0E7FA019B013B0193A5
:1034D000019B002BDED1029B002B03D004930498A8
:1034E0004168084709B030BDE025014C2D03EFE7E6
:1034F00000000111504859368022F8B5964C974B80
:10350000D200002120001C6008F086F92300944AB4
:1035100088331A60934B1A786A23002A00D011333B
:10352000E3620A232365904B37221B780821A363AB
:103530008E4B6018E361102323628D4B3B25636142
:10354000C823DB00A36123008C331A602823013ACF
:10355000E26321646364C267043A201DC2672000ED
:10356000BC3005602000C03001602000C430036022
:1035700020000635CC3005602000083DC8300560CD
:103580002000D03002602200D43211602200D832F4
:10359000136022000226E032200016604222DC3056
:1035A000026020001B3DE43005602000E83001602F
:1035B0002000EC30036023000520F4331860230062
:1035C000F0331A602300183290331A6023009433CA
:1035D000196023001E3A98331A60AF23DB00236082
:1035E000644BFA252363644B6448A3642300B93217
:1035F000FC33FF32AD00A260E56022611D60A06275
:103600007320E0656D386065A065FA2796203F015C
:103610008000E76465625960A0660920E0660020CA
:10362000616757496666E167564E57492667A06746
:103630000F601527676027001A219C373960270023
:103640000731A037396027004B49A837396021007E
:10365000F8310D6021006427A4310F6021005F3F25
:10366000AC310F602100033FB0310F602700B43749
:103670003D00C8272F6027003825B83738609D6087
:10368000424D96215D64424D8900DD61414D1962D4
:103690005D62F53DFF3D9D621E253949DD66596637
:1036A000996499673C49DE651E6618675867D96753
:1036B000BE233A495B00E1508130394BFF30235043
:1036C00004302150C42149006350C623E4205B002C
:1036D000E2500433E2503349334A344BD160344929
:1036E000800019503349E938FF3819503249043005
:1036F000195032493248D16132491163324951631C
:103700001900F4310860CE20304940001160304982
:10371000195019002F48F83108602F49D1658221CE
:103720002E4A89005A501A002D490832D1671A00D2
:103730002C49B432116088212B4A89005A501A0052
:103740002A49883211602A4ADA6408F0BDF801205B
:1037500007F072FFF8BDC0460004FF1FAC5EFF1FFC
:103760009069FF1FA43EFF1F4A0AFF1F3A0700008F
:1037700080C3C9019A02000050C300006A1800000B
:1037800088130000204E0000F009FF1F6509FF1F8D
:1037900068100000C4090000DC05000040420F0072
:1037A00010270000D91AFF1FFC00FF1F0000FF1F99
:1037B0008127FF1FC52AFF1F5D29FF1F251EFF1F31
:1037C0007523FF1F411EFF1FED1FFF1FB11DFF1FB0
:1037D0000124FF1FE924FF1FD918FF1FB923FF1F72
:1037E000C921FF1FD521FF1FB11CFF1F691DFF1F2E
:1037F0009D1CFF1F0223F0B501245E4D5E4E2B7011
:103800005E4B91B01C705E4F03933368002108201B
:10381000FB7006F0E9FD082006F0E0FC002398426A
:1038200005D0FA78552A02D0332A00D096E03360CA
:1038300007F0D2FFFFF760FE1F2201240021514B49
:1038400010AE1A70504B1C70504B1970504B1968C9
:103850009143163A0A431A60602219689143403A2C
:103860000A431A6007F0C0FE07F0F6FEC120FF21F0
:10387000484B80001A588A431A50C5229200985823
:103880008843BF39014399509858434908408021E3
:10389000C9010143802099509958C0050902090ABD
:1038A0000143995080213D48490108F05DF8032308
:1038B00022003B49019400933A4808F0D5F82C22A5
:1038C000394905A808F0E8F805AC61782078023499
:1038D00006F0A4FCA642F8D1344C0020012106F0E9
:1038E000B1FD2268324B03201A40A023DB021343B0
:1038F0002360802322689B041343236022682D4B9E
:103900001A4080239B03134323602B4A2B4B934283
:1039100000D8012007F0F8FE08F066F8802322683E
:10392000DB0413432360287808F0EEF8039B187833
:10393000C0B208F011F808F0BFF82149042007F0E0
:10394000FBFF06F097FE00F0A7F800F0E9FD00F09D
:1039500091FE00F00BFA002011B0F0BD00932100A1
:10396000174A042007F0A8FF8023DB059C62FFF7BD
:103970006DFD5DE74A0AFF1F34F00040A43EFF1FC3
:10398000405CFF1F480AFF1F490AFF1F680AFF1F0C
:10399000BCF0004000E100E0FF00FFFFA83EFF1F79
:1039A0002C51FF1FA84EFF1F08BC001114F000404F
:1039B000FF7FF8FFFFFF9FFF0080FF1F9069FF1F41
:1039C0003B00010870B500252549264A26484D636D
:1039D00008CA1B051B0DED188242F9D10026802272
:1039E000224B92058B630921214B224C1E62224BF4
:1039F0001120DA67214BDA688A43DA609A68204935
:103A00000A409A60266008F0DFF8112007F0FCFEFB
:103A10008022636C93436364EE24E4006C43194A90
:103A2000200C0400642390420AD8FA223300D2000A
:103A3000904205D9144B0A21C01807F08DFEC3B27D
:103A4000124A11201372D48007F0EEFE104B1B783F
:103A5000002B04D10F4B1021187807F0CDFF70BD5B
:103A6000000005408805054000060540FF010000F4
:103A700000F000400038004004E100E03CF000406D
:103A8000FFDFFFFFB70B000030F8FFFF285CFF1FD0
:103A9000625EFF1F605CFF1F002210B51100112045
:103AA00007F08AFE10BD0000F8B500230926374F45
:103AB000374C3B62E3681120B343E36007F0A4FE98
:103AC000112008F081F8112007F0AEFD4023226894
:103AD00080251343236080236268DB021343636005
:103AE000A3682C4A2B43A360A36802211340A36060
:103AF0008023A2689B0113431022A360236C07203C
:103B000093432364236C0F3A1343236480235B00A5
:103B10003B62226B204B1A402263626B1A40626345
:103B2000A26B1A40A263E26B1340E363E3681B4A93
:103B30001340E36006F072FB0121072006F082FCCF
:103B4000174B11205A6C15435D6407F0EDFDFD2104
:103B5000144B154A89005A508023C720626B5B03BF
:103B600013436363E36880003343E3600F4B104A01
:103B700019581140802212020A431A5080229205DD
:103B80001A6008220B4B5A63F8BDC04600F0004093
:103B90003CF00040FFFFDFFFEFFFEFFFFFFF7FFF85
:103BA000003800400000FF1FC539001100E100E0AF
:103BB000FF00FFFF0000054030B503A804880B207C
:103BC000002C0ED14968074D087849780902014355
:103BD0000A20A94205D1012120001980024B1B7A3D
:103BE000137030BD192A0000285CFF1FF7B51500BF
:103BF00008AA16884A680F4F147852781202224396
:103C00000A24BA4214D10122DBB2019200962A00A2
:103C100007F06AFC041E0BD1074B1B68002B07D072
:103C200068782A7800021043424250410130984798
:103C30002000FEBD02290000AC5BFF1F30B501254E
:103C400003790400BFB02B4211D00A49408806F026
:103C5000B7FF28420BD0084B01A95B8D4D800B802C
:103C6000064B00221B7A60880B7104F09FF83FB06E
:103C700030BDC046A45BFF1FD83AFF1F285CFF1F62
:103C800010B50549054806F051FF0421044A0548CE
:103C900006F00EFF10BDC046A45BFF1FFFFF000033
:103CA00034BC0011D83AFF1F10B5024804F000FFE1
:103CB00010BDC0463D3C0011062310B58370103383
:103CC0000371443B43712A3383714433C37100232E
:103CD0000222012103720E4B027041701C88817216
:103CE0004472197A0273C1729A784273DA788273D5
:103CF0000322C2731A7902745A7942740C228274B4
:103D00009A79C274DB7903751123C370152010BD35
:103D1000285CFF1F10B5142007F0F6FD124B14228B
:103D20000021186007F078FD002007F0DDFD01207C
:103D300007F0D2FD022007F0A7FD032004F05CF994
:103D4000042006F071F9052003F09AFB062004F028
:103D500067F8072001F05AFA082006F089FE0920CA
:103D600001F034F810BDC046B05BFF1F07F00CFE39
:103D7000012007F009FD07F06FFE0000094B10B5A8
:103D80000400984205D0012904D12000064906F01C
:103D9000CDFE10BD0229FCD1013904F047FE0028F8
:103DA000F3D0F6E7FEFF0000D65BFF1F70B50D7A7B
:103DB000100004AA2C00168810221440154220D1AD
:103DC000002E20D10A78022A18D14A685178157835
:103DD0000E4A09022943914205D00D4A914209D069
:103DE0001C800A2404E014220A491A8007F054FEB9
:103DF000200070BD0C2208491A80F7E71C800124BE
:103E0000F6E70824F4E70B24F2E7C046F3FF0000CE
:103E1000F4FF0000343DFF1F14BD001110B5040075
:103E20000749084806F082FE074804F081FD00209B
:103E3000E40704D50721054A054806F039FE10BD00
:103E4000D65BFF1FFFFF00007D3D001178BC001115
:103E50001C3BFF1F00B50C4BBFB01A780B4902A8E2
:103E600000F0C2FC6B4680B2D880002809D06A46B8
:103E7000074B01A91B889380064B0022188803F08A
:103E800095FF3FB000BDC046B45BFF1FB55BFF1F91
:103E9000763BFF1F803CFF1F00B50C4BBFB01A786C
:103EA0000B4902A801F0C8FE6B4680B2D8800028FA
:103EB00009D06A46074B01A95B8D9380064B00220F
:103EC000188803F073FF3FB000BDC046DE5BFF1FE4
:103ED000DF5BFF1F1C3BFF1F803CFF1FF7B50E0081
:103EE000377A1C0008AB11003D001A8820231D40C2
:103EF0001F423CD13378022B3BD173681F785B782B
:103F00001B023B431E4FBB4208D01E4FBB4214D086
:103F10001D4DAB4221D00A252800FEBD002A2AD122
:103F2000142C2AD82200F06807F0B6FD174B1C703D
:103F3000012CF1D9FFF7B0FFEEE7002A1BD1202CAE
:103F40001BD82200F06807F0A7FD114B04211C705C
:103F5000104B187807F050FDDEE7E3B20124009221
:103F600001940A00310007F0BFFA0500D4E70825E4
:103F7000D2E70125D0E70B25CEE70D25CCE7C046DB
:103F8000F3FF0000F4FF000002290000DE5BFF1FCA
:103F9000B45BFF1F605CFF1F332310B50400037088
:103FA0000A220749013007F077FD064B0F201B68F6
:103FB0001A0AE37222731A0C1B0E6273A37310BDEC
:103FC000285CFF1F505CFF1F30B5012503790400FA
:103FD000BFB02B4213D00B49408806F0F1FD2842B8
:103FE0000DD06A46084B02A81B889380FFF7D4FFC8
:103FF0006B46D8800022608801A903F0D7FE3FB04D
:1040000030BDC046D65BFF1F763BFF1F10B5024890
:1040100004F04EFD10BDC046C93F001170B516003A
:1040200004AA148805AA15784A6850781178000205
:104030002A4A0843801805284BD807F0C5FC03130B
:104040001E29343F0720042C0BD80522121BAA423C
:1040500000D92A0022491A803000091907F01CFDF6
:10406000002070BD0720112CFBD81222121BAA427F
:1040700000D92A001B491A80EEE707200E2CF0D841
:104080000F22121BAA4200D92A0017491A80E3E71F
:104090000720032CE5D80422121BAA4200D92A00CB
:1040A00012491A80D8E70720032CDAD80422121B01
:1040B000AA4200D92A000E491A80CDE70720032C16
:1040C000CFD80422121BAA4200D92A0009491A801B
:1040D000C2E700220A201A80C3E7C046DCD5FFFFF2
:1040E000C3BC0011FC5BFF1FB3BC0011AEBC0011D0
:1040F000A9BC0011A4BC001110B50D21024A03484F
:1041000006F0D6FC10BDC04698BC00118C3BFF1FCA
:10411000F0B50024274E85B03000B47100F0E2F80D
:10412000254D264BEA89297C9A422FD10423300061
:1041300003AA00F057F90400300000F011F9012340
:10414000B371002C34D16B4699892B68C9BA4B43A3
:1041500029891B4A1B145B1853806B46D9896B68ED
:1041600049BA89B24B4369891B0C5B181548191C65
:104170001BB2834200DD011C0B0400D50021138813
:10418000918001331380200005B0F0BD022722008A
:1041900003AB3000009700F0F7F80E230400297CF1
:1041A0000122300000976B4400F0EEF80443C3E7AF
:1041B0001C00E8E7643CFF1F105CFF1F8305000044
:1041C000285CFF1F0F27000073B5234E300000F05E
:1041D00089F8224D07236A463000297C00F002F955
:1041E00004003000002C33D16B461B787F2B2FD876
:1041F00000F0B6F86B46D878F02302041B031A408F
:104200006B469B8816495BBA9BB21A432B68000920
:1042100053432A891B0C9B184B806B465A789B781A
:1042200012031B011A436B68024353436A891B0C38
:104230009B180C481A1C1BB2834200DD021C13049D
:1042400000D500220B888A8001330B80200076BDC8
:1042500000F086F80124F9E7643CFF1F105CFF1FA3
:10426000285CFF1F0F27000070B5114C237C002B2A
:104270000FD0382B0ED10F4D280000F033F8CC238F
:10428000AC222800217C9B0100F0F4F8280000F00B
:1042900067F870BD084BE2899A42FAD1054D2800B3
:1042A00000F020F800222800217C00F0C5F8EDE79E
:1042B000105CFF1F643CFF1F8305000010B5084B16
:1042C0001A7C002A09D05B69002B06D09847041E8F
:1042D00001D0FEF795FE200010BD0124F9E7C0468D
:1042E000105CFF1F70B5C17905000C00631E9C4176
:1042F0001A4BE402E41849000460C9B2007906F0E0
:10430000D7F8E979687949000131C9B206F0D0F8E7
:10431000E8790930C0B207F087F90023E36661331A
:104320002360AA795B3B002A0ED022689A43023BA5
:10433000134323600A23E3610733236200232363CB
:10434000A3630133E36370BD22689A4302231343DE
:104350002360462363610633A361EFE7005000400A
:1043600070B5002504000368DD66C0790930C0B26D
:1043700007F04AFA2900207906F036F8290060791A
:1043800006F032F870BD0000F8B51E0006AB1D78CF
:10439000002304681700E366616007F05DFA0123FB
:1043A0008022E3662B0027615200013B08D207F010
:1043B0008BFB08200A4A1168002D03D12800F8BDA4
:1043C0002261F2E7236F034203D02369013D33707A
:1043D000013613685B1A032BEED90125EEE7C046C0
:1043E0006008FF1F70B51C00002305681600EB660F
:1043F000696007F031FA01238022EB662300520046
:10440000013B08D207F060FB08200A4A1168002C23
:1044100003D1200070BD2A61F2E72B6F034203D065
:104420002B69013C3370013613685B1A032BEED9FC
:104430000124EEE76008FF1F002370B50468150033
:10444000E366616007F008FA0123E366256107F07F
:104450003BFB8020064A80001168636B034205D154
:1044600013685B1A032BF8D9012070BD0020FCE70C
:104470006008FF1F70B51D00002304681600E36686
:10448000616007F0E9F90123E36626610F33626B8F
:104490001A42FCD02B0A23611023626B1A42FCD013
:1044A000EDB2256107F010FB8020074A80001168FB
:1044B000636B034205D113685B1A032BF8D9012003
:1044C00070BD0020FCE7C0466008FF1F70B51E00ED
:1044D000002305681400EB66696007F0BDF901234D
:1044E000A619EB660F33B4420ED107F0EDFA802027
:1044F0000A4A800011686B6B03420CD113685B1A87
:10450000032BF8D9012070BD21782961696B19420C
:10451000FCD00134E7E70020F5E7C0466008FF1F44
:1045200010B5084CE368002B08D18022064B5202DC
:104530001B689B186360054B1B68236007F0ECFA4F
:10454000A06010BD505CFF1FC8F00040CCF00040E0
:1045500070B5184A936A916A9942FBD116498A68E4
:104560009A421FD39A1A8B60144B0126186893B293
:10457000D202D20E4343424300204C681B0A1B194F
:1045800012029B180E4C0A684B60551CA3420CD8B3
:10459000002801D04B600A600A4A136008680A4B81
:1045A000186070BD581E821ADDE7084A30009B185B
:1045B0002A00EAE700F00040505CFF1F140AFF1FCA
:1045C00040420F00C8F00040CCF00040C0BDF0FFFA
:1045D00070B51F4C23793F2B01D93F2323711D4B0D
:1045E00022791A701878C0B207F0BEFA18231A4957
:1045F0001A4A0B801A4913800B805380A3791949FA
:1046000080200B800C21938001334B43164D191CE5
:104610000001834200D9011C2980D1806379002BDD
:1046200011D101336371237A012B01D80223237244
:104630006279237A0D4853430A21584307F08CF8D6
:104640000B4D286070BDA02BEDD9A023EAE7C04632
:10465000445CFF1F480AFF1F7E3CFF1F503EFF1FA8
:104660007C3CFF1F7A3CFF1F783CFF1F710200005B
:10467000345CFF1FF8B514210020FEF7AFFE114C8B
:10468000011E114D09D10C22104BC1CBC1C4280011
:1046900007F0C2F8FFF79CFFF8BD0C2220000C4980
:1046A000FEF770FE0C2802D0084B43CB43C40C220B
:1046B00028000849FEF766FE0C28EBD00C220021EA
:1046C000E5E7C046445CFF1F105CFF1F08BD0011FA
:1046D000FC0C0000F50C0000F0B51D4C8022A54438
:1046E0000400882069465201400507F05DFA9022D7
:1046F00012016A441300200032C832C316C816C320
:104700008023144C144FA6689B033343A3603B6083
:1047100007F0CAF88823A0685B05C01807F064F8A2
:104720000025882329008022A0685B05C018401955
:104730006944520007F030FA80230135FF355B01F0
:104740009D42EED1A6603E60044B9D44F0BDC04644
:10475000FCEFFFFFC43DFF1F9808FF1F041000007F
:10476000F0B5040087B0002825D0684606F0FCFFAD
:104770001B4C022806D106226946200007F02CF9BE
:10478000002816D06946002301250F262F00E25C81
:10479000013310091030874038002F003240974015
:1047A0003A0002434A610439062BEFD16846FFF70D
:1047B00093FF07B0F0BD182269460A4807F0F4F9E4
:1047C0006A46A300D358013305D01822FF2168465A
:1047D00007F022F8EAE70134062CF1D1E9E7C046F8
:1047E0006509FF1F00090011F0B5002504000E0047
:1047F00085B0AA4200D186E04B1C087801934B7823
:104800008978377909021943F3783F061B040B4373
:104810001F43039720706570252800D196E033D898
:10482000112813D807F058F9690025012501250141
:104830002501AA00B800B1002501250125012501A7
:10484000250125012501250105011F01232800D18E
:10485000DEE0DB2800D02EE1042A00D8ACE01025F1
:10486000052A05D0551F2A003800711D07F014F9DC
:1048700005223100200007F00FF92A003900601DE1
:1048800007F00AF905353EE0562859D010D83328EC
:1048900000D19DE0552839D02628DAD19C4B29003B
:1048A000132218001D0006F0B7FFFEF7A9FB5CE01D
:1048B000712800D177E0722800D180E0602800D113
:1048C0008BE0DC28C5D1022A00D875E07378BFB22E
:1048D0006370B378A370032A05D0033A390092B20B
:1048E000F01CFEF789FC10223900E01CFEF74AFD9F
:1048F000C51C002807DA60705CE00C2220008549A6
:1049000007F0CAF80C25280005B0F0BD013A824D29
:104910000C2A13D8002A0AD02800019907F0BCF805
:10492000FFF756FE0C2228007C49FEF765FC2900A3
:104930000C22601C07F0B0F80D25E4E70C22EBE731
:10494000754D774B2A0043CB43C2E9E7013A704DDE
:104950000C2A11D8002A08D00199280007F09CF8E9
:104960000C2228006F49FEF747FC29001322601C27
:1049700007F092F81425C6E70C22EDE705226A49F4
:10498000601C07F089F80625BDE712226749601C04
:1049900007F082F81325B6E708226549601C07F086
:1049A0007BF80925AFE77178F02905D8614B1888A5
:1049B00001F09EFD0225A6E7FF236370FAE75E4B38
:1049C000012A03D072789A706270F3E79B78F4E75B
:1049D0002000FFF7E1FA050095E7013A564B574DE5
:1049E000062A10D8002A10D00121280059700199F8
:1049F00007F052F801F04EF829000622601C07F07B
:104A00004BF807257FE70622EEE700225A70F3E70E
:104A1000042A04D94A4D2F6007F07EF8A860FFF7FA
:104A200097FD0422039003A9601C07F035F80525C3
:104A300069E7444D062ADFD906222800019906F0CD
:104A4000CBFF0028D8D006220199280007F024F8CF
:104A500006223D492800FEF7CFFB0123364A917814
:104A60000B439370C8E7012AA6D07078FFF778FE51
:104A7000A0E7012800D0ECE6931E344F1A2B04D88F
:104A80007378002B09D100F015F9314B39001D78EE
:104A9000601C6A1E07F000F835E7551E2A000199D0
:104AA000380006F0F9FF2B49AAB23800FEF7A4FB44
:104AB00000F036F9E9E7DA281DD1042A00D87BE7AF
:104AC000082A15D9B37972791B021343F2791204BB
:104AD0001A43337A1B0613433B603B6805223100BF
:104AE0002000039306F0D8FF0422601D03A956E7B7
:104AF000FE236370F1E7DE2800D05DE7511E012A36
:104B000001D10025FFE6019800F0AAFFF9E7C046B1
:104B1000105CFF1F14BD0011445CFF1FFC0C000063
:104B200008BD0011F50C00001C5CFF1FFC5BFF1FA3
:104B3000C83DFF1F803CFF1F405CFF1F243DFF1F3F
:104B4000505CFF1F6509FF1FADAC0000415EFF1FF9
:104B50003F5EFF1FAEDE000070477047020010B5D9
:104B6000094B0A32094C92B2DA815A829881188232
:104B7000207802F023FB0422054B012120781A70D3
:104B800006F03AFF10BDC046523DFF1F8A5EFF1F70
:104B9000895EFF1F013870B5042809D806F014FF9C
:104BA000030928081200234B0221187806F024FF7D
:104BB00070BD204B0821187806F096FF00221E4B8E
:104BC0001A72F5E7802200241B4B1A4D52001A81FD
:104BD00008211A682878DC7206F0E6FD21002878A2
:104BE00006F0B2FF012000F073FE00F053FFDFE794
:104BF000104B0821187806F077FF1048FFF75CF893
:104C00000F4B104A9B79002093800F4A138080221B
:104C1000094B5200D8721A8100F05AFE00F03AFF98
:104C20000A4B9B78002BC3D0094A136006F0ACFFF7
:104C3000BEE7C046605CFF1F345CFF1F893CFF1F5E
:104C4000445CFF1F503EFF1F7A3CFF1F405CFF1F6C
:104C500034F0004010B501290BD1082809D1054BCB
:104C60001B78002B05D02622034B04485A72FFF70D
:104C700075FF10BD625EFF1F345CFF1FC40900009A
:104C80000300F0B50A4D8E18B14202D152008018CF
:104C9000F0BD0C782F6824093C5D0F271C700C7840
:104CA00001313C402F683C5D5C700233ECE7C0464C
:104CB000743CFF1F0E22114B10B51A700D23104CBF
:104CC00010492370093A043B0F48637006F0E4FE74
:104CD0002D2301220D490E48E371FFF7D1FF012278
:104CE0000C49FFF7CDFF01220B49FFF7C9FF002256
:104CF0000A491000FEF780FA10BDC0465E5EFF1F35
:104D00003F5EFF1FC3BC0011415EFF1F6709FF1F0D
:104D1000475EFF1F6609FF1F6509FF1FAEDE00002B
:104D200070B5124C132220001149FEF72BFB114DD8
:104D3000002817DDAB78002B14D0431C2B700923FF
:104D40006B70002300190370287829000130C0B26D
:104D500006F032FF297822000139C9B2002005F09F
:104D6000C5FD70BDFFF7A6FFEEE7C046415EFF1F21
:104D7000AEDE00003F5EFF1F10B5114B1A781870B1
:104D8000002A0ED000280BD10E4B1A78062A07D81D
:104D90005423D340DB0703D50B4B187802F00EFAEF
:104DA00010BD0028FCD0074B1B78012B02D0033B21
:104DB000022BF5D8044B0121187806F01DFEEFE711
:104DC000625EFF1F895EFF1F8A5EFF1F70B5514E36
:104DD000514A52493070082005F02AFC0121022076
:104DE00005F030FB022005F011FC0121002005F048
:104DF00029FB002005F00AFC00F0BAFEFEF700F9DE
:104E000006F04AFD032246494648FFF739FF2D24A4
:104E1000030004221C7044490130FFF731FF3023A6
:104E20000470424D424C437083702E3B062220009A
:104E30004049EB87FEF7A6FA062813D0200006F0BB
:104E400093FC022809D00321200006F0F5FC8D23F5
:104E5000E3706E3B237119336371062220003549DC
:104E6000FEF7CAF9344B1B68FC335C64FFF758FF4C
:104E70000020FFF781FF314C314A0121314B12787C
:104E8000207802F05DF9304A304B1278002120780A
:104E900002F056F901222E4B1A702E4BDB78552B5F
:104EA00031D12D4B3B325A722C4B2D4AAB81EA81CA
:104EB0002B826A822021307806F01EFE01204042BB
:104EC00005F060FD0120404205F0FCFDFFF714F9FC
:104ED000FEF7D6FE00F0A4FC01204042FEF79EFF44
:104EE000012006F001FCF02001F0E6FA0121307803
:104EF00006F082FD307802F0BDFA1A4806F02CFE6A
:104F0000FEF7D2FD70BD6422174B5B7953431A0044
:104F10000A32CBE7605CFF1F594B0011554C001162
:104F2000C83DFF1FFC5BFF1F1C5CFF1F523DFF1FA6
:104F30006509FF1FADAC0000AC5EFF1F8A5EFF1F5E
:104F4000A83CFF1F893CFF1F5E5EFF1F3F5EFF1FE7
:104F5000305EFF1F405CFF1F345CFF1FC409000070
:104F6000CE090000625CFF1F445CFF1FF8B50A0019
:104F700020230D001A40194257D0574B1B78002BA5
:104F800050D0FFF7E5FA554B554C564E996862687C
:104F9000737A8A1ADB039A4202D36160FEF784FDBA
:104FA000327A217A531EDBB2994205D1FFF75CF9C0
:104FB000002000F0A5FD0FE09142F9D300232372F9
:104FC000FFF77CF9012000F09BFD474F3800FEF70A
:104FD00073FE390006F010FE637A002B1FD0013BF0
:104FE000DBB26372002B1AD1404BDB78552B01D119
:104FF00006F0CAFDE37A002B0CD000233C4A3A4F5E
:10500000E3721388380001331380FEF755FE390030
:1050100006F0F2FD642370795843FFF79FFD237A71
:105020000133237220206840F8BD0BB2002B0ADA4E
:10503000304B187806F070FB002801D006F0BCFC5D
:1050400080200002EFE70224214206D0244B0120F9
:105050001A72FFF791FE2000E5E70B071ED5FFF758
:1050600077FA1E4B1E491F4C98684A68637A821A69
:10507000DB039A4202D34860FEF716FDFFF71EF9E4
:10508000FFF7F2F8012000F03BFD00F0E3FB23689E
:10509000DB0701D5FEF7BAFF0820C4E71024214240
:1050A00006D00D4B1B78002BD5D1FEF7FDFDD2E7C6
:1050B0000124214207D0104800F06CF806F09CFA59
:1050C00000F004FDC7E70424080020402142ABD0D3
:1050D000FEF7C0FEBFE7C046625EFF1F505CFF1FC9
:1050E000345CFF1F445CFF1F893CFF1F405CFF1FB7
:1050F000285CFF1F605CFF1F6C3CFF1FF0B51B4B63
:105100001B4F1B883A8804001A4E1B4D85B09A42EB
:105110000DD832889A420AD3184B1A882B889A42A3
:1051200005D1174A174B12881B889A421BD00520BD
:1051300001F018FA3B8802AA13803388019053804B
:105140002B88114D93800F4B02A91B88D3800F4BE6
:105150002A78188802F034FF0D4B08212878019A2C
:105160001C7006F009FD05B0F0BDC0462E5EFF1FA5
:105170007E3CFF1F7C3CFF1F7A3CFF1F2C5EFF1F05
:105180002A5EFF1F783CFF1F8A5EFF1F803CFF1FC7
:10519000285EFF1F13B50C4B1C78002C11D1002882
:1051A00001D00A4B18600A4A0A4B11780A4A107853
:1051B0000A4A01920A4A0092002205F08FFA200062
:1051C00016BD1124FBE7C046895EFF1F245EFF1F4A
:1051D000885EFF1F785EFF1F8A5EFF1F645EFF1FF1
:1051E000685EFF1F10B5064B12201B78052B06D1F9
:1051F000044B13221988044B187801F08FFB10BD63
:10520000895EFF1F803CFF1F8A5EFF1F10B50024D0
:105210000122114B52421870104B1C70104B1A8017
:1052200002F028F904220F4B21001A700E480C32AC
:1052300006F0CAFA102221000C4806F0C5FA07222F
:105240000B4B1C600B4B1C700B4B1C700B4B1A70E8
:105250000B4B1C7010BDC0468A5EFF1F895EFF1F8E
:10526000803CFF1F885EFF1F785EFF1F685EFF1F88
:10527000645EFF1F3E5EFF1F3D5EFF1F823CFF1FFF
:105280003C5EFF1FF8B5174C0600257806A81424CD
:105290000078052D23D1B41F134FA5B21824BD42A9
:1052A0001DD88D1FADB2BD4219D8FA256D00AA4296
:1052B00015D21D000D4F0A3DADB2BD420FD80C4CAA
:1052C00026800C4C21800C4900240A800B4A138054
:1052D000FFF714FF0A4B0421187806F005FC2000A4
:1052E000F8BDC046895EFF1F790C0000750C0000F8
:1052F0007E3CFF1F7C3CFF1F7A3CFF1F783CFF1F5A
:105300008A5EFF1FF0B50BB20D0089B0002B00DBE9
:1053100070E1A44E307806F0FFF9041E50D00378F7
:10532000A22B00D122E1D02B1AD0912B45D143786A
:105330000E2B42D19C4B82889A423ED19B4A836875
:105340001278052A39D1032018567F2835D0984B7A
:105350001B68002B31D05B68002B2ED098472CE0C7
:105360008078072829D806F02FFB0428183F3F74BF
:10537000A8D86378002B0CD101218C4B19708D4B70
:105380001A78002A5BD08C4B307801F0D9FE0028C7
:1053900055D00722854B1A7051E061780029F8D169
:1053A000E378002B11D0854A854B1278307801F0D4
:1053B000C7FE60706378002BEBD1200006F0FCFA8A
:1053C00080200002684009B0F0BD784B1B78022BAA
:1053D000F3D00121307806F0AFF90028EAD101219D
:1053E000307806F009FBE5E76378002BD1D16F4FE9
:1053F000032807D13B78052B02D101333B701EE017
:105400000223FBE76F4B1A886F4B0293002A0BD0E5
:105410001B78002B03D00121307806F0ADFB3B78E0
:10542000062B04D1013BE9E7029B1A70F7E7042B36
:1054300041D10121029B3078197006F0DDFA5C4BF6
:105440001B68002BB9D01B68002BB6D0574A1078C8
:1054500084E76378554F002B27D10622211D5B4836
:1054600006F01AFB62895A4B5A491A80A2895A4B94
:105470001A80E3890B800521397058490A80584AFF
:105480001380228A574B1A80574B1B78012B09D166
:105490001F2001F067F8FA2292004243042130787D
:1054A00006F06AFB0022484B75E7312B00D070E70D
:1054B0000022454B1A700323A0E70622002143482F
:1054C00006F082F90023454A04211380444A3078CB
:1054D0001380444A138006F007FB0821307806F059
:1054E00003FBA379083B5A425341304A03331370FC
:1054F000304B1B78002B06D0334B30781A78002ABB
:1055000006D001F05BFE0122314B52421A8096E731
:105510000121197006F070FAF5E70821307806F0DD
:10552000E3FA6378002B00D047E72C4B2D4F029312
:10553000E388029A04211380294B3078039323894E
:10554000039A138063893B8006F0F6F8002800D0A8
:1055500033E7264B1B68002B00D12EE703990298F6
:105560003A88098800881B68984726E74379132BF7
:1055700000D022E70389012B0AD11D4B1B78022B97
:1055800006D10821307806F0AFFAFFF72BFE14E7BA
:10559000052000F0E7FF08210200307806F0ECFA61
:1055A0000BE7C0468A5EFF1F05140000895EFF1FDF
:1055B000245EFF1FA83CFF1F893CFF1F5E5EFF1F8C
:1055C0003F5EFF1F605EFF1F625EFF1F315EFF1FB9
:1055D000803CFF1F385EFF1F3A5EFF1F2E5EFF1FDD
:1055E0002C5EFF1F2A5EFF1F305EFF1F205EFF1F25
:1055F000285EFF1F8020C001014200D0E2E6CB07F9
:1056000031D5324B1B78002B1DD0314E05AC337891
:10561000052B1AD1023B23702E4B21001B782372DD
:105620002D4B1B7863722D4B187801F02DFD00284F
:1056300009D007202A4B30701B68002B03D01B6851
:10564000002B00D098470120BCE60E20254B0622F7
:105650001B7825492370254B1B78637002ABC0185B
:1056600006F01AFAD8E7022308001840194209D0B8
:10567000174B1B78052B03D11D4B188806F0F4F847
:1056800002209FE60424214203D0FFF737FD2000CB
:1056900098E6082308001840194200D193E6154BFC
:1056A0001C78012C03D0022C0DD008208AE6124B66
:1056B000124A134913481B881288098800880094ED
:1056C000FFF7E0FDF1E7FFF78DFDEEE7625EFF1FFC
:1056D000895EFF1F823CFF1F3C5EFF1F8A5EFF1F2B
:1056E000245EFF1F3E5EFF1F833CFF1F3D5EFF1FCA
:1056F000803CFF1F285EFF1F783CFF1F7A3CFF1F86
:105700007C3CFF1F7E3CFF1F10B502A804880B20C5
:10571000002C10D1496808784978090201430C48E7
:10572000814209D1022119800A4B59881170DB7816
:1057300000205BB2537010BD074C0A20A142FAD181
:1057400002211980034B998811705B79F0E7C046FC
:105750006E2A0000285CFF1F6F2A0000F7B51500B5
:1057600008AA16884A680F4F14785278120222430A
:105770000A24BA4214D10122DBB2019200962A0017
:1057800005F0B2FE041E0BD1074B1B68002B07D09F
:1057900068782A780002104342425041013098470D
:1057A0002000FEBD022900009C5EFF1F30B50125D0
:1057B00003790400BFB02B4225D01449408805F07E
:1057C000FFF928420CD0124B01A95B8D00220B80FF
:1057D00002234B800F4B5B888B80608802F0E6FAD7
:1057E0000D49608805F0ECF9C0070CD50B4B01A9F9
:1057F0001B8800220B8002234B80064B9B888B80EA
:10580000608802F0D3FA3FB030BDC046945EFF1FFF
:10581000AC3CFF1F285CFF1F8C5EFF1F063DFF1F77
:1058200010B5074C0749200005F080F92000064913
:1058300005F07CF90721054A054805F039F910BD46
:10584000FFFF0000945EFF1F8C5EFF1F34BD001140
:10585000AC3CFF1F10B5024803F02AF910BDC0464A
:10586000AD57001170B540253F2608210B4BC207EC
:10587000D2172A40DD789C7835408C432A439C70AF
:10588000DA70820701D521439970400704D5802240
:10589000D97852420A43DA7070BDC046243DFF1FDA
:1058A00013210A4BDA788A43123901400A43DA702D
:1058B0000222104202D0D9780A43DA70400703D599
:1058C0001022D9780A43DA707047C046243DFF1F82
:1058D00010B5054B082419790A00A243002801D00D
:1058E00022000A431A7110BD243DFF1F10B5054B5D
:1058F0002024D9780A00A243002801D022000A43BC
:10590000DA7010BD243DFF1F0821F8B5324D334B2E
:10591000AE7804000E40AE70984204DD67232B7011
:10592000273B6B70F8BD2E4B984203DAE0232B70B7
:105930001A3BF6E700232B706B7083B21A002948DC
:105940005F3292B2284F82422CD9002C03DA5B429C
:105950001CB204232B70053420B20A2105F0FCFE92
:1059600004B2FA239B009C4232DB08232A781343BB
:105970002B706421200005F0EFFE0A2100B205F033
:1059800063FE09B22A787B5C13432B700A21200046
:1059900005F0E2FE0A2100B205F056FE09B27B5C7A
:1059A0006A780AE06970002CDBDA5B421CB20423DF
:1059B0002B70F5226B78092CE8DC13436B700A21FD
:1059C000200005F041FE09B27B5C1E43AE70A9E7E2
:1059D000632CCEDCEDE7C046243DFF1F1B4E0000CC
:1059E0001DFCFFFF2A0800005FBD00110823F7B56A
:1059F000194FCD003E7904001E403E71EDB2632880
:105A000006DD5F3333433B7140231D437D71F7BD9A
:105A10000300093305DA20235B4233433B71C6237D
:105A2000F3E70E4B019300280BDA0423444224B21F
:105A30003B710A21200005F007FE019B09B25B5C67
:105A4000E3E70928F5DD0A2105F086FE019B00B297
:105A50001B5C1E433E71ECE7243DFF1F5FBD001140
:105A6000F8B50A4F05003B780E00002B0CD0084C0F
:105A70002000FEF737FC33002A0020003978FEF7BB
:105A800025FD2000FEF76CFCF8BDC046A05EFF1FA0
:105A90002C3DFF1F70B50A4E0A4D0622310028002A
:105AA00005F09AFF002809D0074C31000622280093
:105AB00005F0F2FF07212000FFF7D2FF70BDC046BE
:105AC000243DFF1F1E3DFF1F1D3DFF1FE62220211D
:105AD00010B50A4B1A70203A5A701C329A70DA7854
:105AE0000A40DA70082219791140033A0A431A7100
:105AF00027225A71FFF7CEFF10BDC046243DFF1F7D
:105B000070B5184B5C78002C2BD1002829D0164D8D
:105B10000A210223E85E05F01FFE00B2FFF7F4FE43
:105B20000423E85E642105F017FE012100B2FFF7AF
:105B30005DFF132220002B7A9A426041C0B2FFF72A
:105B4000D5FE0320FFF78EFE2000FFF7A9FE074BCE
:105B50001878053843425841C0B2FFF7B9FEFFF745
:105B600099FF70BD405CFF1F285CFF1F895EFF1F0F
:105B700070B500250A4C2000A571FEF7B3FB112378
:105B80003E212000074AFEF7A1FCA84200D13E3585
:105B9000054B20001D700123A371FEF7E1FB70BDD2
:105BA0002C3DFF1F4EBD0011A05EFF1F0200F0B58F
:105BB00001270A480A4E51188B1A002B00DCF0BD51
:105BC000082415784308684038404000805B013C59
:105BD00058406D08002CF5D10132EDE7FFFF0000C1
:105BE00070BD0011F0B500250F269D4200DBF0BD11
:105BF0004C5D070944403440A400A058013578406A
:105C0000F3E70000F0B589B06A460D000B000F27DE
:105C1000110010351C780133260024093E4016700F
:105C200054700232AB42F5D12023024AFFF7DAFF6B
:105C300009B0F0BD74BD0011F0B54E780B7889B095
:105C400036020C00170001901E43012A61D9954BC2
:105C50009E4200D877E001339E421CD1062A17D11C
:105C6000CA788B7812021A430B791B0413434A79C2
:105C700012061A438C4B5A6100221A705A808B4AC2
:105C80005A608B4A9A608B4ADA60002009B0F0BDF6
:105C900088225205EEE7884B9E423CD182498B78A0
:105CA000002B00D0F6E00C2A31D10F22A3789343C9
:105CB000E278120213432279120413436279120626
:105CC00013434B60E279A07912020243207A000468
:105CD0001043627A12060243CA60E27AA07A120284
:105CE000024376484A81834208D804236E4914222D
:105CF00001980B7005F0D0FE1420C7E71201D218EE
:105D000089235B059A42F0D801238B70BDE7022AF4
:105D1000FAD00523EAE76A4A01239642E6D1FFF763
:105D200061FA052F0CD9E378A2781B02134322797C
:105D300012041A4363791B061343624A03931360E8
:105D400005F022FFA1E7584D2B78002B9DD1AB78B1
:105D5000002B00D1A0E02B8901339BB20093B3420A
:105D600000D091E0132AD4D9CF7C8B7C3F02122142
:105D700020001F43FFF71AFF874200D08EE0002E5D
:105D80003DD1E378A2781B0213432279E96812041B
:105D90001A4363791B06134303930A228B4212D1E1
:105DA000FF23A370E370237163716B89002B09D10A
:105DB000E37B227C1B0212041343A27B13431B09C7
:105DC00001336B8100226B89002B8ED0002A67D1B2
:105DD000686837013818000B6B690003039098421C
:105DE00005D9686105F000FDEB780133EB70686858
:105DF0001022A11C381805F0CFFE2E8145E76F89CF
:105E0000009A7B1E9BB293423AD1E278A3781202A9
:105E10001A43237905A81B04134362796C681206A0
:105E20001A43EB6800920392211D0C22049305F0A3
:105E300033FE0120260004A940421036FFF7E2FE9F
:105E4000013F012F17D1009A0B232861824200D015
:105E50004CE704221C49200005F09EFE042203A901
:105E6000686805F0A1FEE968039AFF23914200D11A
:105E70003CE7F73B3AE73100FFF7C4FE1036DFE7B7
:105E80000923B742A4D831E7009BB34200D9FCE60E
:105E900007232BE7022329E7032327E7062325E728
:105EA0000A2323E7FFFE0000343DFF1F000001111D
:105EB000FFFF00005048593601FF0000FFFF0011AE
:105EC00002FF000034F00040403DFF1F10B5034CBE
:105ED0000B000122210000F06BFA10BD8D60001153
:105EE0000B8870B506000D000224162B11D92B006B
:105EF0000322094900F05CFA041E0AD1074B2A88E4
:105F00001B88191C934200D9111C300089B200F083
:105F1000EFFA200070BDC046B9600011C65EFF1FD9
:105F200010B54A780400013A0B000220012A07D874
:105F30000A78002A04D005222000024900F038FA2D
:105F400010BDC046E76000110A7810B50B000400D0
:105F50000220002A04D007222000024900F028FA7B
:105F600010BDC046936100110A7810B50B00040003
:105F70000220002A04D009222000024900F018FA69
:105F800010BDC046F961001110B5034C0B000B2287
:105F9000210000F00DFA10BD2962001110B5034C6C
:105FA0000B000D22210000F003FA10BD9B620011CE
:105FB00010B5034C0B000F22210000F0F9F910BDC1
:105FC000F56200110A7810B50B0004000220002AC7
:105FD00004D011222000024900F0EAF910BDC046A9
:105FE00005630011002310B51322190000F0E0F939
:105FF00010BD000010B5034C0B001722210000F06B
:10600000D7F910BD57630011002310B519221900EC
:1060100000F0CEF910BD000010B5034C0B001B22A0
:10602000210000F0C5F910BD91630011F7B5848916
:106030000D0006000121002C22D000238268D356D7
:106040001778002B1EDA0C2C1AD90C3CA4B21319A9
:1060500040880093230002F086FE431E98410130E1
:106060007B06DB0F6B703F23013C1F40A4B22870FE
:10607000AF70AC80002C07D0B3680133AB60002157
:106080000800FEBD0020EBE7AC60F8E70B7803707A
:106090004B8843704B881B0A83700B79C3700420B4
:1060A00070470420022B06D10020537811781B0280
:1060B000009A0B43138070470B8803700B881B0AF0
:1060C0004370022070470420009983420AD153781C
:1060D00010781B0203430B80D37890781B02034394
:1060E00000204B807047F8B50D004B78012400214B
:1060F000461C03702B788B4201D82000F8BD6B78CA
:10610000B01C4F1C012B10D1890069184B8802224A
:1061100033704B88B9001B0A7370691805F094FC42
:1061200004360434A4B2F9B2E4E7122359436B18DD
:106130005A88043132705B8810221B0A7370691808
:1061400005F082FC12361234ECE770B5049D1400A1
:106150001E00052B01D8042070BD637812781B0245
:1061600013432B80E378A2781B02134302226B8037
:106170002A71211D681D063E05F066FCB2B22A8117
:10618000E92AE8D82800A11D0A3005F05DFC0020AE
:10619000E2E7002310B50A789A4201D8900010BDBA
:1061A0009A008A185488013304705488DBB2240A98
:1061B0004470948884709288120AC2700430EAE7AE
:1061C00010B51100029C062B04D004201022142BC1
:1061D00001D010BD022222714B7808781B020343C4
:1061E0002380CB7888781B02034363800431601DD1
:1061F00005F02AFC0020ECE710B50C788B78043110
:106200005C43E4B203702200013005F01DFC601C09
:1062100010BD0420022B06D10020537811781B02F8
:10622000009A0B431380704710B50C000A880231A6
:1062300005F00AFC208810BD70B504000D0004981C
:106240001100012B01D8042070BD1678527812027B
:10625000324302800200F13255701470E125002CA7
:1062600000D10C35023B9AB24280AA42EBD80231EF
:10627000043005F0E9FB0020E6E7042000998342A2
:106280000AD1537810781B0203430B80D37890789F
:106290001B02034300204B80704710B50C000A8896
:1062A000023105F0D1FB208810BD000070B501213E
:1062B0001E000420049C0E400B4218D1CB40DDB2DE
:1062C0008D4214D90A49DBB2098899420FD32300C1
:1062D000EE331D703300580011184978165C09021E
:1062E000314301332152D9B28D42F4D8002070BD20
:1062F0004C3DFF1F10B50C000A88023105F0A4FBCD
:10630000208810BD10B50C788B7804315C43E4B262
:1063100003702200013005F097FB601C10BD10B522
:1063200011000298032B01D8042010BD1478527874
:10633000043B120222430280CA788C781202224364
:1063400042809AB28280EB2AEED80431063005F002
:106350007BFB0020E9E710B50C000B8803700B886D
:106360001B0A43704B8883704B881B0AC3708A8852
:106370000430063105F068FBA088043080B210BDFF
:106380000420012B03D100201378009A137070476A
:1063900010B50C000B8803700B881B0A43704A88E9
:1063A0000230043105F050FB6088023080B210BD2D
:1063B000F0B589B003931E4B029242000700D05AF9
:1063C000019102F020F81325061E2DD0029B012416
:1063D0000370019B002B04D0001903999847001902
:1063E00084B26B461B7A5BB2002B0FDA10213800A7
:1063F00002F01CFB1925002813D130003219E1B23C
:1064000002F066FC051E0CD10C34A4B2042304AACD
:10641000380005A993800696948101F0AFFD051E12
:1064200002D0300005F088FB280009B0F0BDC0465E
:10643000C45EFF1F70B505000C0000280CD00020C2
:10644000814209D010222000044905F0FDFA012004
:106450002B7823736B78637370BDC046B4BD001195
:10646000F0B506000D0017001C0085B002291BD0F6
:106470000020102907D1022B07D0102B03D115E0E3
:106480000020102C08D005B0F0BD69463800FFF799
:10649000D1FF2A0069460BE069463000FFF7CAFFCA
:1064A00022006946380004E0022BE9D12A003900B5
:1064B000300005F039FBE6E7031CF02800D9F02393
:1064C000032008499AB2013A0B80D31703400649CA
:1064D0009B189B100B80D30F04499B185B100B80FB
:1064E0007047C046503DFF1F4E3DFF1F4C3DFF1FF4
:1064F000034B1B888B4202D3024B4000C1527047B2
:10650000503DFF1FC45EFF1F014B4000185A7047EB
:10651000C45EFF1F1722014B1A807047C45EFF1F25
:1065200070B505000E2005F0F7F9041E13D0D02336
:10653000037000230622837007494570033005F07D
:1065400083FA064B2100DA8A62811B7E2373044B97
:10655000187805F0A9F870BDE05EFF1FD05EFF1F40
:10656000A03DFF1F262803D8024B4000C05A7047A9
:106570000148FCE7523DFF1FFFFF000070B5060019
:106580000C00094D1C220021280005F01DF9074BC5
:106590001E70074B1C7005F007FA0123002801D07C
:1065A000002312202B7070BDD05EFF1FA03DFF1F87
:1065B000F15EFF1F70B505000D4C0800E260A160A0
:1065C00010220021656005F027F8012803D1102171
:1065D000A06802F058FD10220021280005F01CF8E8
:1065E000012803D11021606802F04DFD70BDC04646
:1065F000D05EFF1F70B5041E05D1002903D006220E
:106600000D4805F021FA0D4B1D78012D11D1002CFC
:1066100005D102221A7005F037FA280070BD002259
:106620001A70074B1B78FF2BF7D02000FFF778FF7D
:10663000F3E70025F1E7C046E05EFF1FD05EFF1FD5
:10664000A03DFF1F030010B5002801D1002010BDA0
:1066500000780B4A002803D15988D1821B79137620
:106660001378022BF2D10023984200D10333137028
:10667000044B1B78FF2B01D0FFF752FF0120E6E708
:10668000D05EFF1FA03DFF1F002911D000280CD0B5
:106690004B79012803D140225242134303E03F22A9
:1066A0001340032802D001204B7170474022F4E7C9
:1066B0000800FAE770B5094D0100287800280BD0D2
:1066C000074C0622200005F0BFF921002878FFF7CB
:1066D000DBFF200004F0F0FF70BDC046F05EFF1F3E
:1066E000CA5EFF1F00290AD0012808D13F224B793A
:1066F0009343C02B03D0403B5A425341981C7047F0
:1067000070B5174D06002B78FF2B15D00A2005F029
:1067100003F9041E10D0D0230370C83B8370114BC3
:1067200011491B784670C3700622043005F08CF9BD
:106730002100287804F0B8FF0C4B1B78012B0DD1F9
:106740000B4B1B68002B03D09B68002B00D0984795
:10675000084B04211878084A05F026F870BDC04699
:10676000A03DFF1FF05EFF1FCA5EFF1FEC5EFF1F14
:10677000185FFF1F1C5FFF1F60EA0000014B986855
:106780007047C046D05EFF1F014BDB68186870473A
:10679000D05EFF1F074B10B5DA6813680133136032
:1067A000054B1878FF2803D08021C90105F024F992
:1067B00010BDC046D05EFF1FA03DFF1FF7B50E0005
:1067C00002F0C8F8051E1CD00E4B06621F78002F81
:1067D00000D10778AB791020019305F09DF8041ED5
:1067E0000FD0D0230380C73B8370019BE91DC3708A
:1067F0000622043005F028F921003800E66004F094
:1068000053FFF7BD9E3DFF1F014B18787047C046F0
:10681000F05EFF1F054B002805D1054B1A78054B8C
:10682000002A00D1014B18007047C046E05EFF1FF0
:10683000F05EFF1FCA5EFF1F014B58687047C046DD
:10684000D05EFF1F024B1868431E9841C0B27047CC
:10685000F45EFF1F421E03000120152A03D9FF3BEF
:106860005A425341D8B27047F0B51C0000230E00C5
:1068700085B0039002920B70029A934201D30020DC
:1068800019E0E55C5A1CD2B2002DF8D002985119DB
:106890008142F4DC0233DFB2A35C18000193FFF7FE
:1068A000D9FF002807D0013D019A0399EBB233705C
:1068B0008A4202D1E01905B0F0BDDB19DBB2DBE79B
:1068C00010B50C0002F09EF803001220002B03D03C
:1068D0002100588804F010FF10BD000070B50E4D67
:1068E00084006359002B15D0186A002801D004F0E9
:1068F000EBFE2B59586A002801D004F0E5FE2B5915
:10690000986A002801D004F0DFFE285904F0DCFE6C
:1069100000232B5170BDC046005FFF1F1C4B70B59C
:1069200004000E00150099420AD11A4B1B68002B77
:1069300001D1122070BD1B68002BFAD09847F9E7EF
:10694000154B994215D1134B1B68002B0AD01B68BD
:10695000002B07D09847002804D1104B1C70104B17
:106960001D70E7E729002000FFF7AAFF0028E1D10A
:10697000F3E7080001F0EEFF0028DAD003780320E7
:10698000A342D7D12900300004F0B6FED2E7C046BA
:10699000FEFF0000FC5EFF1FFFFF0000F95EFF1F0F
:1069A000F85EFF1FF7B50400808801F0D3FF0025D3
:1069B000A84203D00578A08802F008F81C4E33786E
:1069C000002B1FD0AB421DD11A4B28001978FFF7BE
:1069D00077FF002818D000233370A3790820A77808
:1069E000A688019304F098FF011E0DD0D0230370F8
:1069F000CA3B8370019B477086808371280004F036
:106A000053FE01E0002DE8D1A0880B4B8200D35843
:106A1000002B01D0FFF762FF1721A088FFF768FD68
:106A2000A08801F027FDA08801F0FEFDF7BDC0465B
:106A3000F95EFF1FF85EFF1F005FFF1FF0B587B014
:106A40001D000CAB1B88070001930DAB1B881420A5
:106A500002930EAB1B88160003930FAB1B880091AB
:106A6000049310AB1B88059304F056FF041E1AD044
:106A7000D0230370CB3B47708370C6700622290079
:106A80000430002D11D004F0DFFF019B2100638151
:106A9000029B0098A381039BE381049B2382059BB7
:106AA000A37404F001FE07B0F0BD04F08DFEECE726
:106AB000F7B5009308AB1B8807000C200D001600EB
:106AC000019304F029FF041E13D0280001F042FFB7
:106AD00000280FD00078D0232370C93BA370009BFF
:106AE00021002381019B6770A580E680638104F00B
:106AF000DBFDF7BD014B1878EDE7C046A03DFF1F59
:106B000013B5040064890389C2888188C078009421
:106B1000FFF7CEFF13BD000010B5044C206800281D
:106B200003D004F0D1FD0023236010BD045FFF1FDC
:106B3000A122F0B5818892004A43384B384F1B6838
:106B400004009B189D2292009B18827989B01A60DC
:106B50003B68002B5FD01D78324B1B68002B04D0A4
:106B60005B68002B01D000209847260008363100D2
:106B7000E079FFF7B7FD237DE0710200E078049330
:106B8000638A29000393238A0293E3890193A388EC
:106B900000933300FFF752FFE378002B0BD1E2891B
:106BA000A379A18802920196E2792800009201223D
:106BB00001F0DAFEE0703B68002B20D0FFF7ACFF5D
:106BC000194D287800281AD0184B1978FFF778FE4D
:106BD000002814D02B78E67808200793A78804F0C3
:106BE0009BFE011E09D0D0230370CA3B4670837000
:106BF00087808671079804F057FD00232B701721BA
:106C0000A088FFF775FCA08801F034FCA08801F093
:106C10000BFD09B0F0BD064B9DE7C0463409FF1FD0
:106C2000045FFF1F185FFF1FF95EFF1FF85EFF1F65
:106C3000A03DFF1FF8B5070008000E0001F08AFE16
:106C4000041E18D02620FFF78DFC051E00D12578E4
:106C5000062004F061FE041E0DD00021062204F07F
:106C6000B3FDD0232370C23B21006770A370A680C0
:106C7000E8B204F019FDF8BDF0B585B001930AAB98
:106C80001B78070002930BAB1B7808000D000092E5
:106C9000039301F05FFE061E22D0102004F03CFE9C
:106CA000041E1DD01022002104F08EFD2620FFF7C7
:106CB00059FC002800D13078D0232370C13BA37049
:106CC000009B21002372019B67706372029BA58069
:106CD000A372039BC0B2E3720C9BE36004F0E4FC7C
:106CE00005B0F0BDF7B50D00019001F033FE071EB1
:106CF00020D00E2004F010FE041E1BD02620FFF72B
:106D000031FC061E00D13E78D0232380C53B0622ED
:106D1000A370F91DE01C04F097FE019B2A0063811B
:106D20000123DD401A401D40210022736573F0B23B
:106D300004F0BAFCF7BD0000F0B585B00290100079
:106D40000D0017000A9E039301F004FE041E31D0CB
:106D5000029B002B2ED1039B02795B0724D51223C3
:106D600013430422002E08D10B99002905D10C9958
:106D7000002902D10D9900291AD01A430D9B2271C6
:106D8000002B00D0C9E0002E00D1CFE0002D00D0B4
:106D9000CCE0606A002801D004F096FC1C21300091
:106DA00004F0FAFD606205E002239A430E33D7E750
:106DB00093432371654BBA00D458002C00D1AAE04C
:106DC000002E10D0236A002B03D11C2004F09CFD60
:106DD00020625E4BBA00D358186A002803D01C22E8
:106DE000310004F031FE0C9B002B12D0574CBB003D
:106DF0001D596B6A002B03D1162004F085FD6862D3
:106E0000BB00E358586A002803D016220C9904F0FE
:106E10001BFE0D9B002B11D04C4DBC006659B36A74
:106E2000002B03D1142004F06FFDB0622B59986A37
:106E3000002803D014220D9904F006FE380001F05A
:106E400089FD051E67D0414BBA00D358002B62D094
:106E50001A6A3420002A00D11C389A6A002A01D00C
:106E6000143080B20B9A002A01D01C3080B25B6AC9
:106E7000002B01D0163080B204F04EFD041E4AD023
:106E80001822002104F0A0FC2620FFF76BFB0190E4
:106E9000002801D12B780193D0232370029B20007E
:106EA00063700A23294EA370039BBD00A371AB59E5
:106EB000A780196A1830002905D01C22A06004F0B0
:106EC000C3FD200034307359996A002907D00300AC
:106ED00014221433E060029304F0B6FD02980B9B79
:106EE000002B08D003001C221C330B992061029355
:106EF00004F0AAFD02987359596A002903D016229A
:106F0000606104F0A1FD6B462100187904F0CCFB10
:106F10003800FFF7E3FC05B0F0BD10220D9B0D9982
:106F20001B69A018236204F08FFD2CE70B9B002B3C
:106F300000D13FE7012D00D03CE7606A002801D076
:106F400004F0C2FB1C210B982AE7C046005FFF1F1C
:106F500010B5044C2068002803D004F0B5FB0023D2
:106F6000236010BDF45EFF1F0B4B07B51A68002AA3
:106F700001D100200EBD6946531C01201278073153
:106F8000FFF772FC0028F4D00278012310001840AB
:106F90001A42EED0EEE7C046105FFF1FF0B51F4F5C
:106FA00001203B6887B0002B25D09B78059300F02B
:106FB000B3FB002821D00A20FFF7D4FA04000B20ED
:106FC000FFF7D0FA164B05001E78731E9E413B68F2
:106FD000F6B2191DD878FFF757FB3B682900DA7A1B
:106FE000043303929A7901930292009033002000B7
:106FF000059A04F019FD07B0F0BDFFF7B5FF0028B2
:1070000005D00620FFF7AEFA04000720D8E70820D5
:10701000FFF7A8FA04000920D2E7C046F45EFF1F7C
:10702000F05EFF1F70B50A4E040033780D00FF2B91
:107030000DD0042004F070FC011E08D0D023037092
:10704000CE3B45708370C470307804F02DFB70BD6A
:10705000B03DFF1F70B5040006200D0004F05CFC7D
:10706000011E0AD0D0230370CD3B8370054B4470C2
:107070001B688580187804F017FB002C01D0FFF7FF
:1070800067FF70BDF45EFF1FF8B5264F06003B6832
:107090000D001124002B05D10522234B1B78134230
:1070A00002D112242000F8BD204A10241268002AC0
:1070B000F8D01278002AF5D0DB0719D52B789A1E64
:1070C000012A1AD80C2004F01FFC13243860002871
:1070D000E8D000230A22437029000670023004F031
:1070E000B3FCFFF75BFF041E0AD0FFF731FFD9E7BF
:1070F00000F012FB0028E1D1E4E7002BE2D0D0E75A
:107100000B4B1B78032BCDD11D20FFF72BFA094B1E
:1071100018800028C6D0084B04211878074A04F0CC
:1071200043FBBFE7F45EFF1FF15EFF1F105FFF1F11
:10713000F05EFF1FEE5EFF1F1C5FFF1F60EA000096
:10714000F7B50193194B14001A78052306000F00B8
:1071500012201A4221D0012920D1154B1D68002D83
:107160001BD002201F2C18D8002C02D0019B002B12
:1071700013D0104B1F221E706E1C0021300004F033
:1071800023FB01992200300004F05EFC3100200056
:107190002C70002F06D004F04FFCFEBD064B1220D1
:1071A0001D68DCE704F008FDF7E7C046F15EFF1F4D
:1071B000105FFF1FB03DFF1F0C5FFF1FF8B50F4EA4
:1071C00012243368002B17D01B780F3C834213D155
:1071D00000250B4F0221387804F086FC094B04216E
:1071E00038781D8004F080FC074B28001D80336830
:1071F0005C7004F049FA04002000F8BDF45EFF1F43
:107200001C5FFF1F085FFF1FEE5EFF1F70B50128A8
:1072100023D11B4C2388002B03D01A4A1578002D4C
:1072200007D0194B1B68002B02D01878FFF7C6FF58
:1072300070BD3B2B02D93C3B2380F9E7134E022162
:10724000307804F051FCFA222388920002215A433C
:10725000307804F091FC2580EAE70B4B1B68002B8B
:10726000E6D00B4B1B785B07E2D5084B0221187860
:1072700004F03AFC0022024B1A80FFF769FED7E7C0
:10728000085FFF1FEC5EFF1FF45EFF1F1C5FFF1F08
:10729000F15EFF1FF8B51E4D2868002803D004F0EA
:1072A00013FA00232B601B4E3068002803D004F033
:1072B0000BFA00233360184F05243B781800204058
:1072C000234221D0154800F02BFA3B78234213D0FB
:1072D000202004F019FB2860002813D02022002170
:1072E00004F072FA202004F00FFB041E306005D079
:1072F0002022002104F068FA002004E0286804F04D
:10730000E3F92C601320F8BD00F00AFAF4E7C04658
:10731000105FFF1F0C5FFF1FF15EFF1FA43DFF1FEB
:1073200010B50A4C23681A1E0ED0002808D101306F
:10733000587004F0A9F9002805D02368002B02D06A
:107340000021FFF787FE0122100010BDF45EFF1F31
:10735000F7B5274E050033680191181E21D05C78DF
:10736000244F012C30D1FFF7FFFD002825D020004D
:10737000FFF7F8F80400412814D91F4B02211878B0
:107380001E4A04F011FA1E4B3C3C1C80022233685A
:107390005A703B78002B14D128000199FFF75AFE50
:1073A0000120FEBDFA2292004243002AEED0124B89
:1073B0000221187804F0E0FBE8E7FFF7D3F80200B9
:1073C000F3E700233B70EBE73B78002BE8D1032089
:1073D00004F0A2FA011E08D0D0230370CC3B457004
:1073E00083703368187804F05FF9FFF7B1FDD7E7D1
:1073F000F45EFF1FEC5EFF1F1C5FFF1F60EA0000D2
:10740000085FFF1F10B51749838802008B4220D008
:1074100011D815498B4217D0144900205B1899B236
:10742000012907D8926811785A425341D8B2FFF720
:10743000F9FD012010BD0E4A00209B1807229BB2C7
:107440009A424041C0B2F5E783681878FFF768FFB9
:10745000F0E7836899785A78090218781143FFF7A2
:1074600077FFE7E70A20000006200000F8DFFFFFB3
:10747000AFDFFFFF014B18707047C046B13DFF1FE3
:1074800010B5064C207001F041FA207804F074F930
:107490000521207800F062FD10BDC0461C5FFF1F73
:1074A0000BB273B50D00002B00DBC4E0884B1878DD
:1074B00004F032F9041E0ED00378912B0FD0A22BCA
:1074C00000D1A1E0834B1878FF2852D0210004F0AE
:1074D000EBF800284DD180200002684076BD43784B
:1074E0000F2B76D013D8052B70D00E2BEAD18088C5
:1074F000794B98422BD8794B98421BD8784B9842BD
:10750000E0D1A3681878591CFFF774F838E03E2BD7
:10751000D8D18378032B74D06CD8012B6ED0022B7A
:10752000D0D1704B1B68002B23D05B68002B20D080
:1075300098471EE06C4BC0180C28C3D804F04CF8D8
:107540001DC2C2150BC20B0B0B3223C23C00674B92
:10755000C0180728B6D8664B1B68002B09D01B68DB
:10756000002B06D0200098470AE0A3681878FFF7A0
:10757000C7F8200004F020FAADE7A068FFF762F832
:1075800000289FD0F5E7A3681B78002BF1D0554B5E
:107590001B68002BEDD01B68002BEAD0210055485A
:1075A0009847EDE74F4B1B68002BE2D01B68002B80
:1075B000DFD021005048F3E7504B1B68002BD8D098
:1075C0005B68002BD5D021004348E9E7FFF7EAF9D3
:1075D000CFE780884A4B984203D04A4B984200D06C
:1075E00070E7464B1B68002BC3D05B68002BC0D0F4
:1075F0002100D5E7153B012BBBD963E7FFF798FACC
:10760000B7E7FFF77DFAB4E73F4B1B78042B07D1B0
:1076100000236A4613800179408800F0C5FCA8E782
:10762000364B1B68002BA4D05B68002BA1D0010057
:10763000364898479DE7012421420AD0294B1B6810
:10764000002B04D05B68002B01D00020984701205C
:1076500043E78B070AD5264B1B68002B04D05B68D9
:10766000002B01D020009847022036E70421280093
:1076700008400D4200D131E7254E3388002B21D040
:10768000013B9BB23380002B1AD1FFF7DBF80028B7
:107690000AD0204B1C70164B1B68002B04D05B6873
:1076A000002B01D020009847FFF7C6F8694601F08B
:1076B00001FD6846FEF7FEFF1D20FEF753FF3080F8
:1076C00004200AE7024B187804F00EFAF8E7C046E7
:1076D0001C5FFF1FB13DFF1F0E20000001200000B6
:1076E00009100000145FFF1FFEDFFFFFAFDFFFFF89
:1076F000185FFF1F0C2000000B200000FC5EFF1F26
:107700000D20000013200000F15EFF1FFFFF0000AE
:10771000EE5EFF1FEC5EFF1F10B501F09BF910BD80
:10772000014B18607047C046185FFF1F0B88002090
:10773000162B01D817230420014A13807047C04636
:10774000C65EFF1F00207047074A03001188814270
:1077500007D091880020994202D101308000101892
:1077600070470020FAE7C046245FFF1FF0B58F780E
:1077700006000D00C5B01E2F15D1FFF7E5FF051E51
:1077800003D10024200045B0F0BD00223B003100B1
:10779000C078009200F0B2FB0400A81C00F0D2FBFD
:1077A000FF23EB70EEE7264B062403931B78FF2B99
:1077B000E8D0182FE6D87B08224A013BDB00029272
:1077C0009A589446002ADDD0029AD3185B68002BA1
:1077D000D8D00878002802D14B78012B02D106249A
:1077E000122FCFD107AFAB88697800976446AA689B
:1077F000A047041EC6D1AB78029A5B08013BDB00B0
:10780000D318390030005B689847041E0BD1AB7861
:10781000042BB6D0039A310010782200009700F0B4
:107820006DFB0400AEE76A78002AABD1AA7805A9FF
:107830003B88087130000A704B80FEF747FBA0E7D9
:10784000B43DFF1FC4BD00111D4B37B50500984264
:107850000BD000290AD1FFF777FF002805D119487E
:10786000FFF772FF002800D0058037BD01291AD12B
:10787000FFF76AFF041EF8D001235B420380A37860
:10788000FF2BF2D0FE2B07D00023E07814220093C8
:1078900029001E3300F032FBA01C00F053FB012333
:1078A0005B426380E1E70229DFD1013901F0BEF8D4
:1078B0000028DAD12800FFF747FF041EDFD1D4E704
:1078C000FEFF0000FFFF0000022210B5074B5242EE
:1078D0001A80074801325A809A80DA8000F07EFAD6
:1078E000044801F025F8002010BDC046245FFF1FAA
:1078F0006D770011497800110388F7B50400002B5B
:1079000002D102252800FEBD4268022113782548D5
:107910005268FEF7A5FD00282ED0234F01253A8896
:10792000002AEFD0802321885B0201259B1A99420F
:10793000E8DC0C2003F0E8FF061E31D03B882288EB
:107940009C4600231800019561469DB2491989B2F1
:10795000AA421BD8002801D062443A80002330009C
:10796000082208C0210004F06FF8104A1368002BA9
:1079700013D100251660C5E76268022113780C4810
:107980005268FEF76DFD0028C7D1BAE760681D0197
:107990004019418101330198D6E71A001B68E6E7D8
:1079A0001325AFE732BE0011B23DFF1F205FFF1F5E
:1079B00030BE0011014B18707047C046B43DFF1F28
:1079C00014230A0010B51A40194204D001221021D4
:1079D00001F048F810BD4B06F9D40120884340005F
:1079E000F8E710B514008B0604D50122102101F030
:1079F00039F810BD08230A001A40194202D14BB2CF
:107A0000002B0FDA102101F02DF8002808D02300F8
:107A1000F2331B78002BECD0F1342378012BE8D122
:107A20000020E6E703208907FAD4E2E7F0B51F005B
:107A3000184B85B01C68019002910392002C27D14D
:107A4000200005B0F0BDA5683301ED186B89019ADF
:107A5000934211D3029A93420ED8002F04D10A9B6D
:107A6000002B10D12C00EBE73B002978039A6868C3
:107A7000FEF7F6FC0028F2D10136B6B2A388B34275
:107A8000E1D82468DAE7A3680A9A5B891380E9E7FA
:107A90000026F3E7205FFF1F37B50C000A884988EE
:107AA0000123914217D3002A15D0651D23792A009E
:107AB00002210A48FEF7D4FC102300280BD02379BA
:107AC0006188208800242A000094FFF7AFFF0A2372
:107AD000A04200D0230018003EBDC04632BE0011B7
:107AE00013B50A0008884988012388420BD800286A
:107AF00009D00024137905320094FFF797FF0A2379
:107B0000A04200D02300180016BD13B50A00088853
:107B10004988012388420BD8002809D00024137912
:107B200005320094FFF782FF0A23A04200D0230011
:107B3000180016BDF0B58BB003904A8808880E0077
:107B40000123824255D3002853D00023012704ACDF
:107B500023700022718813000092FFF767FF051E53
:107B60003ED02078002835D12B78022B18D16770B1
:107B70006A8983000130E31880005A806968022214
:107B8000201803F061FF23780133DBB22370042B4C
:107B900019D93B006889013080B2002BD9D01FE091
:107BA00002236370122358436A89231804305A80D1
:107BB00069681022201803F047FF23780133DBB2F5
:107BC0002370002BE5D10C4A6B899B185A42534114
:107BD000DBB2DFE76378012BE4D12B78022BC7D02F
:107BE00022780A23002A04D021000398FEF798F98E
:107BF000002318000BB0F0BD0100FFFF0F4BF0B5E4
:107C000004001868002816D083685D89A54207D84B
:107C10008288AE18B44203DA12019A18934201D155
:107C20000068EFE71E005F891036A74204D10029E3
:107C300000D00D801800F0BD3300EFE7205FFF1F7C
:107C400070B505000C0008880021FFF7D7FF03007E
:107C50000120002B04D022002800197AFFF7C1FE72
:107C600070BDF7B50C00002501902300EE331B78A2
:107C7000AB4201D800200AE06B00E65A0021300038
:107C8000E718FFF7BBFF002802D126800130FEBDB8
:107C9000017A0198FFF794FE002802D03B882380E8
:107CA000F5E70135EDB2E0E710B5040008880021E2
:107CB000FFF7A4FF03000120002B03D02000197A56
:107CC000FFF77EFE10BD0000054B1B68002B01D1A5
:107CD000180004E09A6852898242F6D19888704769
:107CE000205FFF1FF0B50E27002687B0039302AB7D
:107CF000FF183E8005001F4B40891400984207D0B2
:107D00002B78013000976A6880B2FFF78FFE06007B
:107D100002212B7818486A68FEF7A2FB00280FD0D2
:107D20006C892000FFF7D0FF002802D0013C041925
:107D3000A4B2039B002B00D01C80300007B0F0BD24
:107D400002212B780D486A68FEF78AFB0028E7D1EC
:107D500002212B780A486A68FEF782FB002807D0C8
:107D6000002EDED03B88A342DBD17489013CDFE7E3
:107D70006C89DEE7FFFF000032BE001130BE00114B
:107D80002EBE001110B50C00FFF7DEFC0300022030
:107D9000002B0AD0002C00D023609B781720FE2BEC
:107DA00003D00138FF2B00D1002010BD73B50D00AA
:107DB00001A904001600FFF7E5FF172805D0002EE3
:107DC00004D129002000FEF727F976BD01221021F9
:107DD000200000F047FE0028F3D0F6E7014B1860C2
:107DE0007047C046305FFF1F37B56B469D1D0100D1
:107DF00004000222280003F04FFE2B88B02B0ED186
:107E00002379122B09D12300FA331B78012B06D1D9
:107E10000121608800F0E0F801E01B2BF8D037BDAD
:107E200010B5054B0421187000F098F8FFF74CFDD1
:107E3000FEF770FB10BDC046345FFF1F0020F0B599
:107E40000BB20F0087B0834234DA274B187803F067
:107E500063FC051E2BD00378A02B25D103AE310087
:107E6000FEF7E4F8041E0BD1B378DB0724D51F4BD3
:107E700006341B68002B03D0310068889847040043
:107E8000A868002801D003F057FE002C08D1184A3A
:107E9000039B1340174A934206D0B3781B2B03D0A1
:107EA0000121688800F098F8280003F085FD802003
:107EB0000002784007B0F0BD0F4B1B68002B10D0BC
:107EC000310068889847041EDAD07378002BD7D128
:107ED000B27801A90A704B800C716888FDF7F6FF33
:107EE000CEE70624F1E7C046345FFF1F2C5FFF1F7B
:107EF00000FFFF0000011200305FFF1FF7B5019087
:107F0000FC200D0017001E0003F006FD04001320E6
:107F1000002C12D0B02320002370089BF42267703D
:107F2000658026710830002B08D0190003F08CFD05
:107F30002100019803F0B8FB0020FEBD089903F072
:107F400043FCF5E710B5041E06D00078FD2803D8E1
:107F500003F022FCFF23237010BD00000A1F93B220
:107F600010B504000220032B05D882400020024BEC
:107F7000D1529B189C7010BD545FFF1F0B8870B5C9
:107F8000043B04000D000220032B0BD8012120002C
:107F900000F04CFD03001420002B03D0290020002A
:107FA00000F0DEFB70BD000007B51300034A00922D
:107FB0000A00012100F02CFC0EBDC046E581001135
:107FC00007B5019203220092024B0A00122100F031
:107FD00049FC0EBD6382001107B56B4601AA1180F2
:107FE0000449D88008780633012802D1190003F02B
:107FF00083FC07BD355FFF1F0C4B10B518700023C5
:10800000FF210B4A1380138193819380094A538087
:108010001370517293819372D174D3821375517717
:1080200003F02AFB00F0FCF910BDC046645FFF1F9F
:10803000545FFF1F365FFF1FF0B58DB06B46002009
:1080400003910C229B5E834200DBB0E05D4B18780D
:1080500003F062FB051E00D1A4E00378902B00D052
:108060009DE006AF01004688380000F013FA7968F9
:108070000400002900D19CE03B88052B6ED13B8990
:10808000032B1CD905AC200000F0A2F86288172A47
:1080900061D83989131D994231D179682378043127
:1080A0000291D90738D5607800F08EF9071E06D006
:1080B000002303712378012B08D0132B23D0A86849
:1080C000002800D178E003F037FD75E0628802995E
:1080D00009A800F0A6F80290380000F08BF909AA70
:1080E0002378387A0192002231000092029A00F03F
:1080F00012F9380000F064F9029B002BDFD0300049
:1081000000F080F9DBE70378032BD8D1628802996D
:1081100009A800F0D6F8DEE7122B13D1029909A8BE
:1081200000F0B5F8021EEAD127498B88002BC6D093
:10813000887909A92378019161780091310000F0D4
:10814000EAF8BCE7002302AA93833000617809AA09
:10815000FFF72AFFB3E71D4B0993F6E7042B02D084
:108160009A1F012AABD8184A043B9B00995A002950
:10817000A5D0D218907831003A0000F0AEF800286F
:108180009DD13B88042B03D001213000FFF724FF51
:10819000012C04D1A868002801D003F0CDFC2800F0
:1081A00003F00AFC8020039B0002434018000DB03E
:1081B000F0BD012800D182E701213000FFF70CFF5C
:1081C000EDE7C046645FFF1F545FFF1F010017000B
:1081D0000B7803704B784370CB788A781B0213437B
:1081E000438070470A88030002700A88120A4270AE
:1081F0000A88012A06D14A8882704A88120AC27007
:108200000420704702208242FBD14A8804309A70D1
:108210004A88120ADA708A881A718A88120A5A7190
:10822000EFE710B50400012082420CD94B780A78A0
:108230001B0213432380834206D1CB788A781B022A
:1082400013436380002010BD022BFBD1CB788A78CA
:108250001B02134363804B790A791B021343A380EB
:10826000F0E70B8803700B881B0A43704B88837000
:108270004B881B0AC3708B8803718B881B0A437160
:10828000CB888371CB881B0AC37108207047030019
:108290000120082A14D14A780878120202431A8071
:1082A000CA788878120202435A804A790879120201
:1082B00002439A80CA798879120202430020DA8048
:1082C000704710B504000120022A05D100204B7828
:1082D0000A781B021343238010BDF8B50600102056
:1082E0000F00150003F018FB04000120002C0ED035
:1082F000A0230C22290023806780201D002D07D099
:1083000003F0A2FB2100300003F0CEF90020F8BDFD
:1083100003F05AFAF6E7F7B51E00009008AB1420F8
:1083200017001D78019103F0F7FA041E12D0A22362
:108330000370019B47704380099B057146710C22B5
:108340000830002B07D0190003F07EFB21000098B5
:1083500003F0AAF9F7BD099903F036FAF6E737B545
:10836000041E0FD04388002B0CD00025C188132396
:10837000007A172201950095FFF7CDFFFF23658056
:108380006372257037BD000010B50C4904004A889F
:10839000002A09D08B89002B05D00020CB8A02222D
:1083A000834201D010BD012213000A204343002064
:1083B0004032C854C81842800472F3E7365FFF1F8A
:1083C0000023438003707047094B00211A0010B549
:1083D0005C88002C06D01C79844203D10A234B43CD
:1083E000D01810BD01310A330329F1D10020F8E77C
:1083F000365FFF1F10B50400407A03F0CDF9FF236C
:10840000637210BD7047043010B580B203F0B4FA47
:10841000002803D00421494203F03EF910BD0000BA
:1084200070B50025104CA0682580A581A580A842C4
:1084300002D003F081FBA56000250C4C0C4B606D55
:108440001D80230058331D70A84202D003F074FB36
:10845000656500256068002801D003F06DFB0135DB
:1084600008340A2DF6D170BDFC5FFF1FA05FFF1F0F
:10847000F05FFF1F70B5041E09D1054D2880A8814B
:10848000A880A868002802D003F056FBAC6070BD3D
:10849000FC5FFF1FF0B54B8885B00193002343605C
:1084A0000A7905000F00022A00D07BE0CA88032A5F
:1084B00017D98B685E7819783602DC78D8790E4344
:1084C00099781B7A24021B020C43034353495BBA7D
:1084D0000B80331D93421ED1042C04D0631F022B4A
:1084E0000ED9012015E0019A4D4B1201D35A002BF1
:1084F00006D00198FFF7BEFF4A4A136901331361A2
:108500000421B8682E812C80494203F0C5F86860C8
:10851000002005B0F0BD434D042C06D0631F022B94
:108520000FD9EB680133EB60DBE7019A3C4B12019A
:10853000D35A002B05D00198FFF79CFF2B6901331C
:108540002B61374B30000293019B029A1B01019370
:10855000002301998C468B52130063449C80039343
:108560009E81FFF750FF039B041E986016D00421E4
:10857000B868494203F090F8FA880100043A2000F4
:1085800003F062FA0199029AFB888A5A043B9B180D
:10859000029A8B522B6801332B60A2E7AB6901333F
:1085A000AB619EE71E4B0293019B1E01029BF35A97
:1085B000002B2DD002998C19A068002828D0012A00
:1085C00026D1FA889B189BB27352A189994217D37E
:1085D0009B1AC018B96803F037FA029BA289F35AB4
:1085E000934200D07DE700222B81A3882B80A368D3
:1085F0006B60029BF2520B4A53680133536070E781
:10860000084A9368013393600198FFF733FF68E7E6
:10861000044A536901335361F6E7C046665FFF1FA2
:10862000FC5FFF1F6C5FFF1F70B5051E15D10B4C63
:108630000B4B1880230058331870606D002802D04F
:1086400003F07AFA6565250050356068002801D08E
:1086500003F072FA0834AC42F7D170BDA05FFF1F7F
:10866000F05FFF1FF0B51700A12285B092000193C3
:108670004243394B06001B680C009B18D933FF336B
:108680001D78FDF741FF0430854204DD3000FDF721
:108690003BFF0430C5B2BD4207D33A000021300091
:1086A000019B03F0B9F905B0F0BD2900380003F0D3
:1086B000FBF92300C6B250331E700393019B2900BF
:1086C0006365380002F0D0FFCBB20293002B02D0DA
:1086D000039B01361E7000262300503303931B7842
:1086E000B34204D8606D002831D10020DBE7029A44
:1086F0002800002A04D0013B1000B34200D028001B
:10870000F700E719387003F06FFA786000280ED090
:108710003A78019903F098F9019A3B780136D31819
:108720000E4A0193D369F6B20133D361D4E7039BB8
:1087300018706065A74205D1084A1320D36A013337
:10874000D362B0E7606803F0F7F90834F2E703F0AA
:10875000F3F900236365C8E73409FF1F6C5FFF1F4F
:10876000F7B50D0007000421686802F095FF2B891A
:10877000040003702B891B0A43702B8883702B889D
:108780001B0AC3702E8902250436F6B2F42E15D8C2
:108790001B4B9F4214D10C2003F0BEF81135011E73
:1087A0000CD0902303708E3B0371043B4380154B28
:1087B0008460C680187802F077FF00252800FEBD8F
:1087C0005C237B43104AD3180093583301931B78E2
:1087D000002B0FD10300320038000099FFF742FF51
:1087E000019B05001B78002BE8D13800009903F0AD
:1087F00043F9E3E7054A0725536A01335362DDE78E
:10880000FEFF0000645FFF1FA05FFF1F6C5FFF1F84
:10881000F0B587B0009017200F0016000193FFF706
:10882000F2FD1325041E19D00C98031E02D00199E5
:10883000201D9847030AE370052302AAA0700430A4
:10884000908127700098667003A993800494FFF7C5
:1088500087FF051E02D0200003F06EF9280007B044
:10886000F0BD0000F0B587B01F000CAB1B78039182
:10887000059301210DAB06001C78049200F0D6F898
:108880001425002821D02000FFF77EFD0135041EAD
:108890001BD01149059B0A7803700132D2B2131E16
:1088A000C68001D101231A000B7022713000049B95
:1088B00003990097FFF7ACFF051E09D123002100A3
:1088C0000648074A093302F0BFFF280007B0F0BD91
:1088D000002363802370F8E7685FFF1F5F83001148
:1088E00030750000F8B505000E00064C064F2368F1
:1088F000002B02D03100280098470434BC42F6D146
:10890000F8BDC0460C60FF1F2060FF1F0123064A10
:108910005B425380002313715362044A1360536017
:108920009360D360136170472060FF1F0C60FF1FCE
:108930000200002310B506499C000859002801D107
:10894000625010BD0133052BF6D11320F9E7C04664
:108950000C60FF1F034A5388181A43425841404293
:10896000104070472060FF1FF0B585B002930AAB3E
:108970001F780CAB1B88009008000E000192039337
:10898000FFF7E8FF05001120002D1BD10E48FFF76F
:10899000E1FF04001520002C14D006220B99A771CA
:1089A000E01D03F051F8019B30002371029B290068
:1089B0006371009B66802370039B6562E381FFF710
:1089C00091FF280005B0F0BDFFFF000010B5FFF7D4
:1089D000C1FF04000220002C12D060880121FFF7A3
:1089E00081FF606A002801D002F06EFE282200217B
:1089F000200002F0E9FE012300205B426380207129
:108A000010BD000030B5074A074C558801001378A7
:108A10000020A54204D05B1A59424B4158421040F5
:108A200030BDC0462060FF1FFFFF0000084A10B5A0
:108A300001230C00904208D0FFF78CFF031E04D0E6
:108A4000037923405A1E9341DBB2180010BDC04683
:108A5000FEFF0000024B1879431E9841C0B27047D8
:108A60002060FF1F70B504000D001600FFF772FFB5
:108A7000002804D10D4B9C4200D0143070BD416AD7
:108A800003790520002907D012221A40102A02D1AA
:108A90000520002EF2D10F20DB06EFD5897E0C20B9
:108AA000A9428941494249420840E7E7FEFF0000E8
:108AB000030010B5002800D110BD0348034A4188C7
:108AC0009142F9D09847F7E72060FF1FFFFF0000B1
:108AD000002330B5C45CCD5C6C40D4540133102B02
:108AE000F8D130BD0F23002210B5C45C64002243CE
:108AF000CA54C25CD209013BF7D210BD020001008A
:108B000010B52032103102F01FFF10BDF0B58BB050
:108B10000390102005931700049102F0F5FE0090D9
:108B2000102002F0F1FE009B13240190002B05D0D1
:108B300000280CD11324009802F0C6FD019B002BE5
:108B400002D0180002F0C0FD20000BB0F0BD1020D4
:108B500002F0DAFE0600102002F0D6FE1324050013
:108B6000002E00D1AEE0002819D01022002102F022
:108B70002BFE32002900039802F0E6FE041E0ED1FF
:108B800033787F2B51D830000099FFF7ABFF009B63
:108B90001B787F2B53D801990098FFF7A3FF300073
:108BA00002F092FD002D02D0280002F08DFD002C75
:108BB000C1D1102002F0A8FE0600102002F0A4FE91
:108BC0000290002E7CD0002878D03A000F3223008B
:108BD0000125121105D00F333B4015B25A425341C3
:108BE0001BB26A1E1201002B33D0049BD2B298181C
:108BF0000099029AFFF76CFF013D1022002130001E
:108C000002F0E2FDADB2049F2D017D19AF4242D0CA
:108C1000002C33D0300002F057FD029B002B00D116
:108C200089E7180002F050FD85E729003000FFF7C2
:108C300059FF28002549009AFFF74AFFA7E72900B6
:108C40000098FFF74FFF28002049019AFFF740FFE7
:108C5000A5E70F210F4004998A18D9B28F4208D98D
:108C6000D15C06A819540133102BF6D1029A019950
:108C7000C0E7791A48424141C901F2E739003000A2
:108C800006AAFFF725FF3200039806A902F05CFE52
:108C900010370400BAE7002CBCD13000029906AAB4
:108CA000FFF716FF320006A9039802F04DFE0822D6
:108CB00004003100059802F0C7FEABE71324A9E7D2
:108CC0001324AAE7002800D06EE733E738BE00116E
:108CD000F0B58BB00F0016000225009000283FD0A1
:108CE000002A3DD00B1DDBB21800029302F00CFEEF
:108CF0001135041E34D0FDF747FD05003A000099F8
:108D0000201D02F081FCEBB20393E3702B0CDBB26D
:108D10002F0A00936370FFB22B0E2370A77001938C
:108D2000FDF72CFD1022010006A802F06DFC2100C9
:108D3000029A04AB06A8FFF7E9FE051E0DD1039BBE
:108D400008223370009B04A9B370019B7770F37005
:108D5000301D02F059FCFDF71DFD200002F0B4FCAF
:108D600028000BB0F0BDF0B58FB00D00149E03903D
:108D700004920593002A03D1022420000FB0F0BD15
:108D8000002EF9D00398FFF7E5FD1424071EF4D058
:108D90007278337812021A43B3781B041343F278C3
:108DA00012061A43036A0192934201D30133E3D1BD
:108DB000002D03D03B7901249B07DED5082200213A
:108DC00006A802F001FD059B13240433DBB2180052
:108DD000029302F099FD051ECFD0059A0499043044
:108DE00002F012FC04223100280002F00DFC3900D0
:108DF000102210310AA802F007FC2900029A06ABE3
:108E00000AA8FFF783FE041E0FD1082206A908A8AE
:108E100002F0FAFB0822311D08A802F085FE0128A5
:108E200007D101990398FDF7C9FC280002F04CFC1A
:108E3000A3E70124F9E7000070B51C4C0500236886
:108E4000181E10D0002D14D11A78002A0CD1981CAD
:108E5000083202F0F9FD02F00FFD0135002808D1BB
:108E600023681D70012070BD0A331800082202F02B
:108E7000EBFD2368002BF5D0122002F04DFD061EFD
:108E80000DD0C123216803704570023110220230D9
:108E900002F0DAFD23683100587802F005FC206802
:108EA00002F012FC00232360DCE7C0464860FF1F8D
:108EB000F8B504002020FDF755FB0D4EA700BB5967
:108EC0000500002B0DD000280BD0D878FF2809D141
:108ED00008492A000C55F35907480333611802F07A
:108EE000B3FCF8BD290002F067FB0028F0D1F8E7D9
:108EF0006460FF1F4C60FF1F09A1001170B5064D93
:108F000084006359002B05D0D87802F045FCFF227D
:108F10006359DA7070BDC0466460FF1F70B506000B
:108F20008CB00C00150000213022684602F04CFC89
:108F300031001022684602F067FB1D202100032249
:108F4000684402F061FB6846FFF7D8FD2D2104005C
:108F500003222800694402F057FB20000CB070BDCA
:108F6000F0B50700160097B001931CAB1D783022B6
:108F70001EAB00910AA800211C7802F025FC1022EB
:108F800039000AA802F040FB1022002102A802F0DA
:108F90001BFC0722310002A802F036FB072202ABBD
:108FA0009818631E9C41019902F02EFB02AB9C7342
:108FB0002B005A1E934102AAD3730021102206A847
:108FC00002F002FC06221D9907A802F01DFB1A20E0
:108FD00002ABC01806221F9902F016FB102200995E
:108FE0000EA802F011FB102202AB0EA908781C7823
:108FF000013A6040D2B2087001330131002AF5D144
:109000000AA8FFF77BFD102212A904000EA802F0A7
:109010001BFD102206AB0EA908781D78013A6840A6
:10902000D2B2087001330131002AF5D10AA8FFF746
:1090300065FD044310222098E4B212A902F0E4FA7C
:10904000200017B0F0BD70B50E0014008CB0010008
:10905000102268461D0002F0D7FA3100082204A849
:1090600002F0D2FA2100082206A802F0CDFA6846E2
:10907000FFF744FD04001022280008A902F0C4FAFA
:1090800020000CB070BDF8B506000D0000243719A3
:10909000AC4200D3F8BD02F047FC030A3B70631CEE
:1090A000DBB201379D4203D90234F054E4B2EEE75B
:1090B0001C00EDE773B506000C000225002819D04E
:1090C000002917D0032101A8FFF7DDFF6B469A792D
:1090D0003F231A40013313436A463000937101A9BC
:1090E0002200FFF71BFF051E04D10322E01C01A98B
:1090F00002F0AAFC280076BD03785807DA08C00FF2
:10910000D20080009B0710439B0F1843C0B27047EA
:1091100007230B40C908C9000B43037070470000C8
:1091200070B50400FFF7EAFE134DA4006359002B4D
:1091300021D0186A002801D002F0C6FA2B59986E87
:10914000002801D002F0C0FA2B59D86E002801D0B7
:1091500002F0BAFA2B59186F002801D002F0B4FAC5
:109160002B59586F002801D002F0AEFA285902F0AE
:10917000ABFA00232B5170BD6460FF1F0E4B8000C3
:10918000C35870B50C00002B0FD09D68002D0CD07B
:109190002B78201D0B706B784B70A97CFFF7B8FF04
:1091A0002B7E23726B69E36070BD102200212000CA
:1091B00002F00AFBF8E7C0466460FF1F014B18602D
:1091C0007047C0466060FF1F074A03008000825856
:1091D00010B5002A06D0D088984203D1012901D1C8
:1091E000FFF79EFF10BDC0466460FF1FF0B5264E1E
:1091F00095B087000B93BB590500099112200A9284
:10920000002B31D0D888FFF7A5FB04001420002CD8
:109210002AD0280010A9FFF7B1FFBB591E781D6A9C
:10922000002E23D00895FDF7EFFA07000020FDF788
:10923000F1FA0790A379E61D069310AD0CA90898E2
:1092400000F0E2FA0EA9280000F0D7FA0B9B0A9969
:109250000493069B09980293079B0396019300973A
:109260000EAB0CAAFFF77CFE15B0F0BDFDF7CCFAF3
:1092700006903000FDF7CEFAE31DA779079310ABF7
:1092800006000893DAE7C0466460FF1F30B50C4C57
:1092900085002A59030085B00120002A0ED018004D
:1092A0006946FFF76BFF2B591A78D888054B002ABF
:1092B00000D1054B6A46072100F0D9FB05B030BD4F
:1092C0006460FF1FFB9700110998001130B5094C2D
:1092D0008500295985B010226846253102F0B4FB7B
:1092E0002A591121044BD0886A4600F0C0FB05B012
:1092F00030BDC0466460FF1FA598001130B5094C11
:109300008500295985B010226846353102F09CFB52
:109310002A591121044BD0886A4600F0A8FB05B0F9
:1093200030BDC0466460FF1FE3980011F7B54D4F94
:1093300086001020F4590D0002F0E6FAF35920627D
:10934000186A132200286CD0033A29009C6802F0A6
:109350007BFBF3591A780192002A58D11E6A227DAC
:10936000317B944651400122019F114201D1674651
:109370001740217D914339432175377B4F40BC46CF
:1093800060460027800701D44F08174001210220C2
:109390008F40227D82433A432275377B5740BC463B
:1093A00060460027400701D497080F400420227D23
:1093B000BF0082433A432275627D0027944660468F
:1093C000727B42400A4201D167460F400121627D13
:1093D0008A433A436275777B5740BC466046002714
:1093E000800701D457080F400220627D7F0082432E
:1093F00017436775767B00227E40760701D4BA0852
:109400000A400426617D9200B1430A4362756A787E
:10941000002A08D06278002A05D005220533DA77C1
:1094200000221000FEBD04222979114205D1A17C41
:10943000114202D10533033AF1E7019A21782C78E1
:10944000002A02D10A002100140018220429E8D8B9
:10945000042CE6D805206043034A05331218525CF9
:10946000DDE7C0466460FF1F48BE001110B50A006A
:109470001121024B00F0FBFA10BDC0463F990011CC
:109480000B0030B587B001AD2B806B460400110096
:10949000981D082202F0D8FA2A000B212000024B66
:1094A00000F0E5FA07B030BD6799001110B50A0069
:1094B0001121024B00F0DBFA10BDC046BB99001130
:1094C00013B50B0011006A4613706B4604000622A8
:1094D000581C02F0B9FA6A4608212000014B00F03E
:1094E000C6FA13BDDB99001110B50A001121024B19
:1094F00000F0BDFA10BDC0462B9A00117FB50500E3
:109500000B4BAA00D4580800002C0FD0666F237FA5
:10951000E28821780396266F0296E66E0196A46E85
:109520000094FDF709FC2800FFF7FAFD7FBDC04657
:109530006460FF1F10B51721FFF7E0FF10BD0000AA
:1095400070B50A000D00064B0221040000F08FFAEE
:10955000060029782000FFF7D1FF300070BDC0461B
:109560000B99001170B586B000236A4613708368AA
:1095700004001D78681E0A2859D801A902F024FAAF
:10958000060633373B3F43474B4F5300180000F06C
:1095900042F9062312284BD000281BD16088FFF720
:1095A000D9F90823002813D04279002A47D1264B45
:1095B0001A78072312070BD5244B1A680723002AB1
:1095C00006D01668002E03D0290001AAB047030078
:1095D0006A4613706B461B786088002B2AD1FFF710
:1095E00067FC06B070BD180000F06CF9D4E71800F5
:1095F00000F087F9D0E7180000F093F9CCE71800E5
:1096000000F0ADF9C8E7180000F0C3F9C4E718008E
:1096100000F0F6F9C0E7180000F0F6F9BCE7180012
:1096200000F013FAB8E7180000F013FAB4E70723C4
:109630006A46137069466088FFF782FFD1E7052309
:10964000012AC5D1024BB8E7F15EFF1F5C60FF1F26
:109650006060FF1FF8B52C4F8600F35904000D0021
:10966000002B40D0DA8882423DD15A78062A33D185
:109670001A78002A2ED0012099681A6A097D0142C1
:1096800006D0157B054203D007225A700120F8BD91
:109690000220014204D0157B054201D00922F4E7E3
:1096A0000420014204D0127B024201D00B22ECE7DD
:1096B000164B1B68002BE9D05B68002BE6D020001E
:1096C0009847BB5900215B78122BDFD12000FFF7B0
:1096D00015FFDBE70E4BECE7112A04D1002900D07F
:1096E00032252900F2E7002D08D12000FFF732F9DA
:1096F000002803D0102302791343037121002800AE
:10970000FDF798FAC2E7C0466460FF1F5C60FF1F68
:109710006060FF1F70B50E4E8500AB590400002B32
:1097200013D01B78002B11D10A4B1B68002B04D0DF
:109730005B68002B01D02000984773595B78122B8F
:1097400003D100212000FFF7D9FE70BD024BECE7EA
:109750006460FF1F6060FF1F5C60FF1F094B80009B
:10976000C3581020002B0CD01A6A002A09D09B681D
:10977000002B06D0127A1B7E101C9A4200D9181CAE
:10978000C0B270476460FF1F70B503000D00140085
:109790000220002A30D000292ED013700B78081D2B
:1097A00053704B789370FFF7A7FCE0700120022103
:1097B0002B7A23716B7B034063716A7B0A401343EE
:1097C000042263716E7B1640334363716E7BF6082F
:1097D000F600334363712B7B0340A371287B014068
:1097E00000200B43A371297B0A401343A3712A7BFA
:1097F000D208D2001343A37170BD10B50A00010056
:109800000120FFF7C1FF10BD10B50A0001000220C2
:10981000FFF7BAFF10BD70B506000C000220002E45
:1098200030D000292ED07378201D0B70B3784B7088
:10983000F178FFF76DFC01223579257271794B10B3
:1098400008001340934010400343881010408000EC
:10985000C9080343C9000B436373B1794B10080077
:109860001340934010400343881002409200C908FF
:109870001343C9000B4321202373FCF773FE854279
:1098800001D2122070BD2220257AFCF76BFE8542A2
:10989000F7D823781820042BF4D86378012BF1D85B
:1098A0000020EFE7030010B50220002909D0002BAB
:1098B00007D00322481C0A7019000D3202F0C4F8C8
:1098C000002010BD03000222080010B5002B06D0B6
:1098D000002904D00E32591C02F0B6F80022100004
:1098E00010BD030010B50220002909D0002B07D0BD
:1098F0000422481C0A7019000C3202F0A5F800205E
:1099000010BD10B5FFF7DEFF10BD030002200029D7
:1099100006D0002B04D0052200200A701B784B7063
:10992000704703000220002B08D0002906D05B7886
:1099300000200B70013B082B00D918307047030042
:1099400010B50220002909D0002B07D00622481CA0
:109950000A7019000A3202F077F8002010BD10B525
:10996000FFF7B0FF10BD02000B00022010B5002968
:109970000ED0002A0CD00721197011885970118857
:10998000090A997011180822D81C02F05DF800200D
:1099900010BD03000A00022010B5002B0CD00029D6
:1099A0000AD099785878090201431180901CD91C7B
:1099B000082202F049F8002010BD030010B5022073
:1099C000002909D0002B07D00822481C0A70190072
:1099D000921802F039F8002010BD02000B0002209E
:1099E00010B500290BD0002A09D00921197011786F
:1099F00018185970511C062202F026F8002010BDDC
:109A000010B5FFF75FFF10BD02000B00022010B57C
:109A1000002A09D0002907D05178197011180622A0
:109A2000581C02F011F8002010BD030010B50220F0
:109A3000002909D0002B07D00A22481C0A701900FF
:109A4000063202F001F8002010BD10B5FFF73AFF12
:109A500010BD02000B00022010B5002A06D000291C
:109A600004D018005178FFF753FB002010BDF0B56B
:109A700085B017001E006A46062305000800918184
:109A80009380FEF7C0FC1324011E02900CD0380016
:109A9000B047041E05D1280001A9FEF76FFA041E85
:109AA00002D0029802F048F82800FFF701FA2000DF
:109AB00005B0F0BDF0B504008BB001911500002198
:109AC000102202A801F080FE334EA700B8590028EA
:109AD0003CD0C388A34239D10378002B36D14278D9
:109AE000062A18D102000100553235310C3006AB80
:109AF000FFF7A9FA002829D12000FFF72FFE020066
:109B000006A902A801F0A0FF200002A901F05CFD57
:109B100001200BB0F0BD816E002917D00B8A112AED
:109B200028D19D420ED101981231093A01F0FCFF73
:109B3000012807D1BB5920009D6EFFF70FFE2900B9
:109B40000200DEE732212000FFF7D8FC2000FEF7FC
:109B500001FF061E1BD0416A002918D00B8AAB42B8
:109B600015D108220198123101F0DEFF01280ED133
:109B7000716A0AE09D42E9D108220198123101F090
:109B8000D3FF0128E2D1BB59996E8A7EB9E7200044
:109B900001F0DAFDBCE7C0466460FF1FF0B56B4D15
:109BA00087007E5985B0337802900393002B00D054
:109BB00087E0B368346A01937078062817D10122D0
:109BC0001B7D134202D0217B114218D10222134285
:109BD00002D0217B114251D10422134203D0237BB6
:109BE000134200D08BE0019B5A7DEB5991E007387E
:109BF0000428F8D801F0E8FE032E42678300B36E14
:109C0000002B03D11C2001F07FFEB066EB599C6E47
:109C1000002C1CD010220021200001F0D5FD02985C
:109C2000FFF79CFD01002000FFF72DFA01F07CFEFC
:109C30002082200008211230FFF725FA0298FFF752
:109C40008DFDA076EB592100D888FFF70FFC082284
:109C5000EB591CE0B36E002B05D01A00198AF0886E
:109C60001232FFF70DFC0222019B197DEB591142C4
:109C70003DD0207B10423AD0073208E0F488FCF750
:109C8000DBFD01002000FFF711FC0A22EB595A709E
:109C9000029B9C002A595378073B042B11D8D0888B
:109CA000FEF758FE00284ED0C3895A08D21828491A
:109CB000029B0298CB542B5941180433254801F0DC
:109CC000C3FD05B0F0BDFCF79FFD030001208342FA
:109CD00001D100200393EB59DE88FCF79BFD03992B
:109CE00002003000FFF7ECFB019AEB59117D0422D2
:109CF00011420CD0217B114209D00B22C7E7F68814
:109D0000FCF73CFD01003000FFF7EEFB6BE7019A2A
:109D1000527D01210A4204D0607B084201D00C220E
:109D2000B5E702210A4204D0607B084201D00E222E
:109D3000ADE704210A4204D0627B0A4201D010221E
:109D4000A5E71222A3E7FA225200B0E76460FF1FE2
:109D50006860FF1F13A1001110B5064B1A78042389
:109D6000100018401A4200D00348FFF727FA0020DD
:109D700010BDC046F15EFF1FB83DFF1F70B5040067
:109D8000FFF7D4FA051E43D12000FFF77FFA234ED8
:109D9000A400A0598268937CDB0708D50321036ADD
:109DA0001B790B40012B02D1017F0B430377431D2D
:109DB000D97F8B1E022B0DD8022900D00121C0882B
:109DC000FCF790FF042133591A7F59700A431A7720
:109DD000280070BD01290CD10223102243700021FC
:109DE0000C3001F0F1FC305910213530FFF74BF900
:109DF000EEE70529ECD10223D118437010220C3074
:109E000001F022FE04233259117F0B431377EAE756
:109E100008251828DCD1053DDAE7C0466460FF1F3D
:109E2000F0B58BB0059143887E4F9E00F459150024
:109E30000493002C15D1012902D000200BB0F0BDF5
:109E4000101D57781678FFF757F9EB683200029328
:109E50002B7A0499019300903B002000FCF70CFF43
:109E6000EBE7E388049A934201D00820E6E72378E1
:109E7000012B00D1D4E0059B581E092800D9CFE062
:109E800001F0A2FD05CE0A29CC506C859AB22900BA
:109E90000498FFF773FFD1E7200029001022453016
:109EA00001F0D2FDB9594B78042B02D1013B4B7024
:109EB000C3E70B000A00253335320C310498FFF755
:109EC00095F90498FFF702FA0522431E9841BB5901
:109ED000C0005A70B2E7200029001022553001F06E
:109EE000B3FD049B4F4C9D00295904980A0006AB12
:109EF00055320C31FFF77AF929591022453106A85D
:109F000001F012FE012808D10498FFF7F7F9059037
:109F1000002804D106222B595A7005988EE7082391
:109F20000593FAE763780C2B7AD1E36E002B03D10B
:109F30001C2001F0E9FCE066BB59D86E00286FD008
:109F40001022290001F080FDBB590498DC6EFFF758
:109F500005FC0D22A076BB595A706EE7E06E002812
:109F60005ED063780D2B5BD12B8808220382A91C5D
:109F7000123001F069FDBB599A68517D02221142ED
:109F800026D0186A407B104222D00C32E4E7637876
:109F90000E2B45D1236F002B03D1162001F0B4FC0A
:109FA0002067BB59186F002803D01022290001F048
:109FB0004BFD0F22BB59CFE763780F2B30D1206FB9
:109FC0000622691C103001F03FFDBB599A68517D93
:109FD0000422114203D0196A497B1142D5D10021D4
:109FE0000498FFF78BFA28E7636F002B0DD0BB595D
:109FF000586F0028F3D01022290001F025FD01221E
:10A00000BB5952425B6F1A61E9E7142001F07CFCF6
:10A01000BB5960675B6F002BE9D126E72978DFE742
:10A0200007200BE76460FF1F10B5064C207001F09D
:10A03000E3FB06212078FDF791FF0348FEF778FC4B
:10A0400010BDC0467760FF1FC991001100200BB200
:10A0500070B50D00834216DA264B187801F05CFBD0
:10A06000041E0DD00378922B0ED0A02B37D0224B9C
:10A070001878FF283AD0210001F016FB002835D1CE
:10A0800080200002684070BD43780E2B0BD03E2B21
:10A09000EDD18378052B12D0082BE8D18179808807
:10A0A000FFF7D8FA08E0154B82889A42DFD183681F
:10A0B0001878591CFEF7C0FE002817D1D7E7104BBF
:10A0C0001B785B0712D50F4B1B68002B0ED09B68CB
:10A0D000002B0BD0C289811D80889847ECE7FFF7E1
:10A0E00041FAA068002801D001F026FD200001F00F
:10A0F00063FCC5E77760FF1FB13DFF1F182000001C
:10A10000F15EFF1F6060FF1F10B50078FFF712FAC5
:10A1100010BD10B50078FFF7FDFA10BD0C234343C6
:10A12000084A10B59B185A68002A03D0012901D1AA
:10A13000904710BD9B68002BFBD00029F9D19847B0
:10A14000F7E7C0469460FF1F01238340094A10B51A
:10A15000946B1C439463506B98435063D46B200002
:10A160009843012901D120001843D063116B0B43A0
:10A17000136310BD00800040F0B500240127154B8B
:10A1800085B0DA6B144E03921A6C0192DA64019B6B
:10A19000E3403B4217D0039DE5403D400295E5B2C8
:10A1A00002992800FFF7BAFF316A736A002908D0C4
:10A1B0003900002B01D0029979402800FFF7C4FF35
:10A1C00001E0002BF9D101340C36172CDFD105B09A
:10A1D000F0BDC046008000407860FF1F064B0121A3
:10A1E0005A68C2400A4204D01B68C34018000840A5
:10A1F00070471B6DF9E7C046008000400122064B06
:10A200008240002903D0D9680A43DA607047D968D0
:10A210009143D960FAE7C0460038004030B50324C6
:10A2200044430F4BE25C1B199C785D7801232D1B86
:10A230000135AB40013BA340A140DB430C00122899
:10A2400007D808499200521811681940214311603B
:10A2500030BD054A11680B4023431360F8E7C04640
:10A260008FBE001108F0004014F00040C21F70B50E
:10A27000D4B20623092C0BD80125084C954000299F
:10A2800008D00021FFF7CAFF23682B432360002377
:10A29000180070BD2368AB43F8E7C04600380040A3
:10A2A000214BF0B51B185B78022B21D103244443CA
:10A2B0001E4A1F4EA35C1219947801221500854096
:10A2C000B76B013CE4B23D43A240B563194C122880
:10A2D00015D89B0000290CD117495B1899680A43CF
:10A2E0009A600123205C154A834011680B43136078
:10A2F000F0BD11495B18996891439960F1E70E4BE5
:10A3000000290DD159690A435A61225C1328E8D00B
:10A310000123203A93400A49086803430B60E7E7AA
:10A32000596991435961F0E77860FF1F8FBE0011B2
:10A3300000800040D4BE001100F00040A0F00040BA
:10A34000A4F00040F8B500241B4E1C4D1C4B1B5DB7
:10A35000012B1FD1194A9269E2401A420BD0012207
:10A36000B25693402200143AD2B2022A09D81549B3
:10A370004A6913434B61013402360C35172CE5D181
:10A38000F8BD0022B2560F499200521891680B4353
:10A390009360F0E7022BEED1E7B23800FFF71EFF23
:10A3A00001235840C1B23800FFF77AFF3800FFF7A9
:10A3B00015FF6877DFE7C04661BE00117860FF1FB8
:10A3C0007960FF1F00F00040012202388240054BF7
:10A3D000002903D059690A435A617047596991436A
:10A3E0005961FAE700380040F8B50E0001210F006E
:10A3F0008740114A0400D368FD43BB43D360831EEA
:10A400008B4201D8FFF7E0FF00212000FFF72EFF6D
:10A410000A4A0B4B5168012E05D139431B19516073
:10A420005E700020F8BD2940516002221C19627044
:10A430009A6915409D61F4E70038004000800040B3
:10A440007860FF1F012210B58240074B002906D01B
:10A4500019680A431A600121FFF7C6FF10BD196889
:10A4600091431960F7E7C046008000400C2370B5A7
:10A47000002543430A4A29009B181D70094B04001C
:10A480001B185D70FFF7B0FF0123A34006492800A9
:10A490000A681A430A6005490A689A430A6070BD4F
:10A4A0009460FF1F7860FF1F3480004030800040C0
:10A4B00070B504000E00FF2813D003250540FFF7F8
:10A4C000D5FF084AA3089B009B183F22ED00AA4035
:10A4D000AE40196820009143314319600121FFF714
:10A4E0008DFE70BD18380040F8B50C244443134B62
:10A4F0000500E4186368002B03D1A3681220002B29
:10A500001AD0022201270E4B00215B195A70280035
:10A510002770FFF769FF63681E1E08D0A3683E001E
:10A52000002B04D02800FFF759FE4640F6B2280061
:10A530003100FFF709FE0020F8BDC0469460FF1F00
:10A540007860FF1FF7B5C420FF222B4B80001958FD
:10A55000002491433F3A0A431A508022274F520267
:10A56000274E1A60274B1D5D002D21D0A31E012B05
:10A5700003D80121E0B2FFF727FF012D18D11F4BAF
:10A580009B69E3402B4213D0E3B218000193FFF71D
:10A5900025FE01000198FFF755FFE3B2143B022BA3
:10A5A0001DD801217156184A8D405369AB43536140
:10A5B0003B7F002B0DD0E5B22800FFF795FF280068
:10A5C000FFF70CFE7B7F0100834202D02800FFF7DB
:10A5D000A5FD01340C370236172CC3D1F7BD01217C
:10A5E00000237156F3568D40074A9B009B189A68CA
:10A5F000AA439A60DCE7C04600E100E07860FF1FF4
:10A6000061BE00117960FF1F00F0004010B501210C
:10A610000400FFF7E9FE0123044A002011194B70E2
:10A62000A34091690B43936110BDC0467860FF1F42
:10A6300070B50E0015000400FFF718FF0C236343EC
:10A64000094A20009B189D605E60FFF74DFFF021D6
:10A65000064B074A8900051E5A5002D02000FFF71A
:10A6600005FF280070BDC0469460FF1F0000FF1F5B
:10A6700079A1001170B5134D07202C78002C1FD143
:10A68000982221005200280001F0C6F80123C420BE
:10A69000FF222B700C4B80001C635C630B4B1C6017
:10A6A0005C600B4B195891433F3A0A431A50802281
:10A6B00052021A600D20074A074901F07DF8200078
:10A6C00070BDC0467860FF1F00800040A0F00040D1
:10A6D00000E100E045A5001145A3001170B51D0083
:10A6E00002240C2910D8094ACA40D2070CD5FBF71E
:10A6F00045FF041E08D1059A04992800FBF75AFF6C
:10A70000FCF7C8FDFFF728FB200070BD1210000009
:10A7100030B50D7802232C009C43184201D02B4306
:10A720001C0008252300AB43284201D02B00234303
:10A7300020241D00A543204201D01C4325002A23CC
:10A740000D70184204D011781E3B0B43137030BDBE
:10A750000028FCD10C2113788B43F7E7F8B51D00D6
:10A7600006AB1B88140007AA0E000B201778002BDD
:10A7700027D10A78022A49D14A6850781178000214
:10A78000244A08438018042840D801F01DF9031218
:10A790001D1B2300F06801F037F9021CC0B2B8425B
:10A7A00000D93A1CD2B22000F1682A8001F04CF99D
:10A7B00006E00222F3681B882A8023701B0A63705C
:10A7C0000020F8BD0622EEE701232B80F3681B78FA
:10A7D0002370F5E7F368002B16D008222A801A8828
:10A7E00022701A88120A62705A88A2705A88120A55
:10A7F000E2709A8822719A88120A6271DA88A271CC
:10A80000DB881B0AE371DBE72B80D9E701202B8073
:10A81000D7E7C04600D6FFFFF7B516000A781D003F
:10A8200008AB1F880C000123022A18D14A6850780F
:10A83000117800022B4A0843801803280FD801F032
:10A84000C3F802254439E06801F0DEF8C0B20723FE
:10A85000B84204D37B190193152B02DD0D23180098
:10A86000FEBDE0682A003100C01901F0EDF86B462A
:10A8700000209B88E268D0541B4B1B68834203D0A6
:10A880001B68834200D098470023E8E70B23002F82
:10A89000E5D1022DE2D1737832781B021343E268CE
:10A8A0001380114B1B68002BEED01B68002BEBD0E4
:10A8B0000120E8E70B23002FD1D1062DCED12A00AD
:10A8C0003100E06801F0C0F8DEE70B23002FC6D1AD
:10A8D000012DC3D132787533012AC0D8E3681A70CC
:10A8E000D2E7C04600D6FFFF8462FF1F70B50C00A0
:10A8F0001500072837D801F067F8041436361B36E0
:10A90000242E182015290BD8184E162200213000AD
:10A9100000F05AFF22002900300001F095F80020D5
:10A9200070BD18200229FBD11288114B1A80F6E75E
:10A9300018200829F4D10A000E48290001F0ACF8CB
:10A94000EDE718200129EBD10B4B10780B49DA69A0
:10A95000FFF7DEFEE3E718200129E1D1064B10786E
:10A960000749DA6BF4E70220DAE7C0466C62FF1FA2
:10A970005A3EFF1F503EFF1FE03DFF1F083EFF1FD6
:10A98000283EFF1F030010B50020DB0704D5072178
:10A99000024A034800F08CF810BDC046ECBE00111E
:10A9A000E03DFF1F054A03001068002803D082889D
:10A9B0009A4201D1806870470068F6E77C64FF1F07
:10A9C0000A88030008009A4204D08A8804309A4218
:10A9D00000D0002070470000F8B5F22200230D4F90
:10A9E0000D4E7968050042433370994200D07B6078
:10A9F0000A4C0021200000F0E7FE00231A007C60D2
:10AA0000AB4202D100203370F8BD01332280DBB2AB
:10AA1000F234F5E77465FF1F7265FF1F8064FF1F46
:10AA200073B56B4601900600684615001980FCF767
:10AA300063FF041E11D1002D0FD07689002E11D096
:10AA40000C2000F061FF00280ED0084A0460136853
:10AA500086808560002B02D11060200076BD1A0030
:10AA60001B68F7E70224F8E71324F6E77C64FF1F6E
:10AA7000012100220A4B10B549420A4C19809980E5
:10AA80009A719A70084B2070012019805A60FFF764
:10AA9000A3FF2078FCF78EFF0448FDF749FF10BDA7
:10AAA0008C62FF1F7C65FF1F7465FF1F5DAB00118B
:10AAB000022310B5002802D0FFF7B2FF03001800F0
:10AAC00010BD0000030010B50020DB0704D50421F1
:10AAD000024A0348FFF7A4FF10BDC04600BF0011A3
:10AAE000603EFF1FF0B50E2687B003930CAB1F88A6
:10AAF00002ABF6180500080031000292FDF77EF85F
:10AB000004000120002C0FD03088FFF74BFF03001A
:10AB10000E20002B08D05E68002E05D021002800F2
:10AB2000039B029A0097B04707B0F0BD0A4B10B5DF
:10AB3000984207D10122002352420A808B708A80FA
:10AB40008B7110BDFFF73CFF0028FAD001235B4258
:10AB5000038000238370F4E7FFFF0000F8B50500D1
:10AB600001290AD1134E00243388F227AB4219D0B1
:10AB700028001149FFF7DAFF06E0022904D1013964
:10AB8000FDF754FF0028EDD0F8BD3B006343726829
:10AB9000D018D35A002B09D03A00002100F014FE3F
:10ABA0000134E4B2054B1B78A342EED801235B428B
:10ABB0003380DDE77465FF1F8C62FF1F7265FF1F26
:10ABC00010B5FFF7FDFE03000020834200D0987807
:10ABD00010BD0000F0B589B01C000EAB80CB039017
:10ABE0001E8810AB1B78049202930B7A0D00DB06D3
:10ABF00016D42B780593022B24D00498FFF7D2FEAD
:10AC0000002812D003689C46002B0ED0029B220025
:10AC1000019329003B00644603980096A04705E095
:10AC20000498FFF7BFFE002802D10E2009B0F0BD46
:10AC30008368002BF9D00A2229000398984700283E
:10AC4000D7D0F3E76B6858781A786B4B0002104343
:10AC50009842D2D8043B984210D2684B984242D0D6
:10AC600015D8674BC0180128C7D80B20002EDDD19E
:10AC7000EB681A7859683A80200028E0614BC018C8
:10AC8000032800D979E000F09FFE846A789E5E4B2D
:10AC90009842B2D10B20002EC8D101233B80EB6833
:10ACA00031001B7823706889013080B2FCF7A6FF61
:10ACB0003A88031E0ED0017802328A183A804289FF
:10ACC00062704289120AA27059680278E01C00F092
:10ACD000BBFE06E004323A8031000422601C00F022
:10ACE00073FD0020A2E70B20002E9FD1EB6807A97F
:10ACF0001E8804233B80330A300026706370FCF703
:10AD00007DFF051E28D004AB9A890E2304A95B1889
:10AD10003E49C668FCF7E6FF00280BD12B783C487B
:10AD20006A680599FBF79CFB002803D1012304AA5C
:10AD30005B42D3813278022A06D17168201D00F06F
:10AD400083FE3B8802333B800E2304AA9B181B889A
:10AD5000A3701B0AE370C4E704ABDE81F4E70B20A9
:10AD6000002E00D062E7E9680398FFF729FF02236D
:10AD70003B802070000A6070B3E70B20002E00D0EB
:10AD800054E70222EB681B883A8023701B0A637029
:10AD9000A7E7E86800F038FEC2B203000720B2421D
:10ADA00000D243E70DD00299DBB27118994202DB61
:10ADB000921BD3B20293029BE9681A003B80891967
:10ADC0005AE70023F6E70B20002E00D02EE70722DB
:10ADD000EB683A801A7822705A7862705A88A270AA
:10ADE0005A88120AE2701A792271DA886271DB8855
:10ADF0001B0AA37175E7C046042900000228000061
:10AE000000D8FFFFFFD6FFFF03280000FFFF000070
:10AE100030BE0011F0B58DB06B46002008912022A5
:10AE20009B5E83423DDAA64B187800F075FC071E46
:10AE300032D00378B02B2CD10079023816281FD8D5
:10AE400000F04AFE17001E001E001E0031001E000A
:10AE500096001E001D011E0052011E0073011E00FF
:10AE6000CD011E0050021E001E001E008E021E009C
:10AE7000E302944B94491B8878880B80FBF730F8E9
:10AE80003800FCF7B1FF914B1B68002B01D0380054
:10AE90009847380000F090FD8020089B0002434056
:10AEA00018000DB0F0BDEE220021874800F08CFCA8
:10AEB0000BAA3B7B7989388900923A000D32FCF766
:10AEC000B5FD0400804B1B78002C3FD146E0804B41
:10AED000788805937F4B4100CB5A0BAE073BDBB222
:10AEE00032880293002301937B4B21000693009349
:10AEF000059BFFF76FFE744D002810D1069B3A8A20
:10AF00001B889A420BD138000599123000F00CFED4
:10AF1000002804D02B7862899B00EB185A801623F6
:10AF200006A81B18328820007989FCF7DBFE2B78F5
:10AF300004009A00AA1851880029C3D00133DBB25B
:10AF40002B70002807D006A9C98A9180634A12880D
:10AF50009A42BCD802E0012149429180002B04D0E2
:10AF600059497888FAF7F0FF8AE73E890A2479E0A0
:10AF700000253E89574B06937B88069A5B009B5AB7
:10AF8000033B9D4202DB002DF0D05BE0162206A8B9
:10AF900012183B7B798900923A0030000D32FCF7A1
:10AFA00045FD0590002858D04689017A7888FCF73D
:10AFB00007FD041E44D1464B78880793069B410049
:10AFC000C95A454B0439C9B206AAD28A06930291DE
:10AFD000019400930599079BFFF7FCFD041E2FD1F8
:10AFE000069B39491A88931C002D26D14B807988FD
:10AFF000384B4900CB5A5119033B8B4220DD059B4E
:10B0000031485B8941190B71A91C0135C9B2EDB2F8
:10B01000059145191B0A2B71059B2D4904331818FE
:10B0200000F012FD2C4B059A1B88D318DDB22C4B77
:10B030009E4205D00136B6B29CE749889942D6D0E7
:10B04000002D0CD0204C2800618800F085FB20707A
:10B0500021007888FAF788FF12E7059CF0E7002CBA
:10B0600000D183E77B78142B00D109E716493B799F
:10B070004E800B700C717888FAF728FF00E71624D1
:10B0800006ABE41821003889FCF7B8FD011E00D199
:10B09000B7E1788822880F4C45002C5B0A4D013CB3
:10B0A000E4B2029400240F4B01940095FFF792FD47
:10B0B000041E00D014E129007888FAF765FFDFE666
:10B0C0007C65FF1F503DFF1F9462FF1F8862FF1FBA
:10B0D0008863FF1FC45EFF1F7864FF1F4E3DFF1F84
:10B0E000FFFF00009662FF1F162406ABE418210044
:10B0F0003889FCF783FD011E00D182E1788822881F
:10B10000AE4C45002C5BAE4D013CE4B202947C8910
:10B11000AC4B01940095FFF75DFD041E00D0DFE00D
:10B1200029007888FAF73AFFAAE60025A44B1D808B
:10B130003B00F6331B78A24A78880792AB4208D9C5
:10B140009E4B12880693069943005B5A013B9A4234
:10B1500003DB0799FAF72CFF92E616246B00FB1825
:10B16000059306ABE418059B21001889FCF746FD02
:10B17000011E03D1059B01241E8973E77888924B39
:10B180002288069C099343001B5B904E013BDBB277
:10B190000293002300960193099BFFF71BFD041EF9
:10B1A00002D0059B1E895DE77B88069A5B009B5A4F
:10B1B000079A108832881218934202DC1B1A013B4E
:10B1C00033807F4C023032880999001900F03CFC32
:10B1D0002388328801359B182380EDB2A8E70BAA9B
:10B1E0003B7B7989388900923A000D32FCF71EFCCE
:10B1F00000250590059B002B04D10A24002D00D1C9
:10B200006EE060E0059B7888197AFCF7D9FB0100B5
:10B21000041E63D1694C6C4B788806940993069B95
:10B220004400E45A694B063CE4B20BAE3288079303
:10B230000294019100930599099BFFF7CBFC041E32
:10B240004CD1079B5E491B881A1D002D30D14A80C6
:10B25000059B5B4C5A8963191A716B1C9BB2E318EE
:10B26000120A1A71162306A832881B1879890598C4
:10B27000FCF738FDFF21AA1C2E1D03350B0005909D
:10B2800092B2B6B2ADB2002803D006ABDB8AD9B217
:10B290001B0AA218651911712B714C4D301D2A889B
:10B2A0004949201800F0D0FB2B88F618B5B2A1E769
:10B2B0004988914207D17A8806995200525AEB1870
:10B2C000053A9A42C4DC3E4C2800618800F0ECFB51
:10B2D000207021007888FAF775FED1E5002DF2D1B3
:10B2E0003E89BFE6162606ABF61831003889FCF712
:10B2F00085FC3D000400FA3500282DD0037A9B061A
:10B300000CD400227B893989788800923A000C326B
:10B31000FFF7E8FB041E10D03E8915E03088FFF7E8
:10B3200041FB00281AD08368002B17D0210012227D
:10B3300078889847041EE4D0EEE72B78002B02D1E2
:10B340007888FAF74FFE00262B78002B00D097E57F
:10B35000002C00D194E585E60124DDE70E24DBE72F
:10B36000162506ABED1829003889FCF747FC041EAA
:10B3700047D0037A9B0611D4154A7B8811889942DD
:10B3800003D01448814207D11380134BF2261D7855
:10B390000023D9B2A94221D30924A1E72888FFF7C5
:10B3A00001FB00282FD08368002B2CD02100122213
:10B3B00078889847041EDFD092E7C046C45EFF1F1E
:10B3C0009462FF1F9662FF1F8863FF1F7864FF1F50
:10B3D0007465FF1FFFFF00007265FF1F31005943B6
:10B3E000546801336018615A0029D2D13C000834F6
:10B3F0002100F22200F028FB21007888FAF7FAFDFC
:10B400003EE501246CE70E246AE71D4B1A887B8811
:10B410009A4231D07888FAF7F7FD31E5F2230598A2
:10B4200051684343CD18C95A00291FD03B7A012BDC
:10B430000BD16C88AB887888AA1D0094FFF752FB6B
:10B44000041E02D000233B722E88F2220021280025
:10B4500000F0BAF900232B80059B0133DBB2059382
:10B46000084B05991B78064A8B42D7D801235B42CB
:10B470001380002CCED0F5E5002634000596EFE7CA
:10B480007465FF1F7265FF1F70B504000E00150084
:10B49000FFF796FA031E08D131000548FFF790FA2E
:10B4A00003001120002B02D01C8000209D7070BD75
:10B4B000FFFF0000F8B50B4F06003B780D001400AD
:10B4C000FF2B0ED00A2000F027FA011E09D0B1236D
:10B4D0000380002346800371C5800481387800F022
:10B4E000E3F8F8BDA13EFF1FF7B50F0008A906005D
:10B4F000088809A90B240988002821D10234022BCD
:10B500001ED1557813782D021D432B008B430193D8
:10B510007334002B14D1FB68300019000093FFF73F
:10B520004FFB019C85420BD02A0030000099FFF7A9
:10B53000ABFF041E04D12A0030007989FFF7BAFF5F
:10B540002000FEBDF0B50E7885B003900AA80588EE
:10B550000120022E0DD14C682778647824023C43E8
:10B56000054FBC4205D10398DBB201960095FFF769
:10B57000BBFF05B0F0BDC04602290000034B10B56B
:10B580001B68002B00D09847FEE7C0468065FF1F70
:10B5900007B501A8FFF7F2FF044A05480021121A77
:10B5A00000F03AF9F8F726F9FEE7C0468465FF1F78
:10B5B000A43EFF1F0000000001B40248844601BC05
:10B5C000604700BF5147010001B40248844601BCF6
:10B5D000604700BF311B000001B40248844601BC33
:10B5E000604700BF3936FF1F01B40248844601BCE2
:10B5F000604700BF3935FF1F01B40248844601BCD3
:10B60000604700BFC51D000001B40248844601BC6C
:10B61000604700BF4551010001B40248844601BCA7
:10B62000604700BF1D4B010001B40248844601BCC5
:10B63000604700BFA533FF1F01B40248844601BC28
:10B64000604700BF456B010001B40248844601BC5D
:10B65000604700BF350E000001B40248844601BCBB
:10B66000604700BFE528FF1F01B40248844601BCC3
:10B67000604700BF090E000001B40248844601BCC7
:10B68000604700BF7918000001B40248844601BC3D
:10B69000604700BF691F000001B40248844601BC36
:10B6A000604700BF5549010001B40248844601BC0F
:10B6B000604700BF594F010001B40248844601BCF5
:10B6C000604700BFC521000001B40248844601BCA8
:10B6D000604700BF014C010001B40248844601BC30
:10B6E000604700BF6571010001B40248844601BC97
:10B6F000604700BF6DBC000001B40248844601BC35
:10B70000604700BF8D12000001B40248844601BCAE
:10B71000604700BF212DFF1F01B40248844601BCD1
:10B72000604700BFF54E010001B40248844601BCE9
:10B73000604700BFF92AFF1F01B40248844601BCDC
:10B74000604700BFC94A010001B40248844601BCF9
:10B75000604700BF091B000001B40248844601BCD9
:10B76000604700BF350E000001B40248844601BCAA
:10B77000604700BF6D33FF1F01B40248844601BC1F
:10B78000604700BF5D17000001B40248844601BC59
:10B79000604700BFA54F010001B40248844601BCC8
:10B7A000604700BF1147010001B40248844601BC54
:10B7B000604700BF5952010001B40248844601BCF1
:10B7C000604700BF812BFF1F01B40248844601BCC3
:10B7D000604700BF154D010001B40248844601BC1A
:10B7E000604700BFC9A9000001B40248844601BCFB
:10B7F000604700BF6532FF1F01B40248844601BCA8
:10B80000604700BFC926000001B40248844601BC5D
:10B81000604700BFE533FF1F01B40248844601BC06
:10B82000604700BFB70E000001B40248844601BC67
:10B83000604700BF392BFF1F01B40248844601BC9A
:10B84000604700BF055E000001B40248844601BCA9
:10B85000604700BFA946010001B40248844601BC0C
:10B86000604700BF75A9000001B40248844601BCCE
:10B87000604700BF2526000001B40248844601BC91
:10B88000604700BFD91B000001B40248844601BCD8
:10B89000604700BF2146010001B40248844601BC54
:10B8A000604700BF792EFF1F01B40248844601BCE7
:10B8B000604700BFB130FF1F01B40248844601BC9D
:10B8C000604700BFC56D010001B40248844601BC59
:10B8D000604700BFADAE000001B40248844601BC21
:10B8E000604700BF3D18000001B40248844601BC17
:10B8F000604700BFB14E000001B40248844601BC5D
:10B90000604700BFE117000001B40248844601BC53
:10B91000604700BF3D4B010001B40248844601BCB2
:10B92000604700BF1D4D010001B40248844601BCC0
:10B93000604700BF2951010001B40248844601BCA0
:10B94000604700BFBD30FF1F01B40248844601BC00
:10B95000604700BFE548000001B40248844601BCCE
:10B96000604700BF9134FF1F01B40248844601BC08
:10B97000604700BFB54C010001B40248844601BCD9
:10B98000604700BFE928000001B40248844601BCBA
:10B99000604700BFED4A010001B40248844601BC83
:10B9A000604700BFF94C010001B40248844601BC65
:10B9B000604700BF5125000001B40248844601BC25
:10B9C000604700BF434D010001B40248844601BCFA
:10B9D000604700BF4D36FF1F01B40248844601BCDA
:10B9E000604700BFF30E000001B40248844601BC6A
:10B9F000604700BF492DFF1F01B40248844601BCC7
:10BA0000604700BF0D52010001B40248844601BCEA
:10BA1000604700BFDD52010001B40248844601BC0A
:10BA2000604700BF5118FF1F01B40248844601BCA3
:10BA3000604700BF851F000001B40248844601BC76
:10BA4000604700BF4D1F000001B40248844601BC9E
:10BA5000604700BFE94C010001B40248844601BCC4
:10BA6000604700BF8552010001B40248844601BC12
:10BA7000604700BF4550000001B40248844601BC45
:10BA8000604700BF7D18FF1F01B40248844601BC17
:10BA9000604700BF291C000001B40248844601BC75
:10BAA000604700BF810E000001B40248844601BC1B
:10BAB000604700BF090E000001B40248844601BC83
:10BAC000604700BFE12AFF1F01B40248844601BC61
:10BAD000604700BF9DA9000001B40248844601BC34
:10BAE000604700BF6136FF1F01B40248844601BCB5
:10BAF000604700BFB352010001B40248844601BC54
:10BB0000604700BF0124000001B40248844601BC24
:10BB1000604700BFEDA5000001B40248844601BCA7
:10BB2000604700BF156B010001B40248844601BCA8
:10BB3000604700BFCD4C010001B40248844601BCFF
:10BB4000604700BFD949010001B40248844601BCE6
:10BB5000604700BF2124000001B40248844601BCB4
:10BB6000604700BF3555000001B40248844601BC5F
:10BB7000604700BFDD66010001B40248844601BC95
:10BB8000604700BF8B52010001B40248844601BCEB
:10BB9000604700BF0D35FF1F01B40248844601BC59
:10BBA000604700BFB131FF1F01B40248844601BCA9
:10BBB000604700BFE130FF1F01B40248844601BC6A
:10BBC000604700BF5522000001B40248844601BC12
:10BBD000604700BF2534FF1F01B40248844601BC02
:10BBE000604700BF5933FF1F01B40248844601BCBF
:10BBF000604700BF017F000001B40248844601BCD9
:08BC0000604700BF056A000067
:10BC08000001010302000303040305020602070200
:10BC1800080209020A030B030C020D000E030F03AE
:10BC2800100311001300140315001600B93B00118E
:10BC3800ED3B001100000000020000004ABC0011AA
:10BC4800192A0F180A000000F1590000FD2400000D
:10BC580041460100398000114DA00011A174001166
:10BC68003D7E00110553001115AE00116D4F0011F6
:10BC7800AD3D0011DD3E0011000000001616000069
:10BC88000200000094BC0011F4FFF3FFD2FC000096
:10BC98001D4000110000000000000000547579618B
:10BCA8000042312E340030303139006769746875CC
:10BCB800622E636F6D2F7076767800544830354663
:10BCC8000000000002000000E0BC0011292A282A18
:10BCD800272A262A252A242A0A180000E204000016
:10BCE8007102000078EC000074400000102700008A
:10BCF80060F0000006640000204E00000000000014
:10BD0800050000001F501D00023CB400000119008E
:10BD180014000000A10200003031323334353637C8
:10BD28003839414243444546000000000957001194
:10BD38005D57001100000000020000004CBD00111A
:10BD48006F2A6E2A1A18EAD8BC80F0FC600000003E
:10BD580000000000000000F505D39727B6F615F798
:10BD6800B777E6F0C7F27200000001A000000000FB
:10BD78006410B71DC8206E3BAC30D9269041DC76E4
:10BD8800F4516B6B5861B24D3C7105502083B8ED8E
:10BD980044930FF0E8A3D6D68CB361CBB0C2649BB2
:10BDA800D4D2D38678E20AA01CF2BDBDFB349B5FD7
:10BDB800800000800010000000000000A360001157
:10BDC8002D770011C7600011357B00114B61001100
:10BDD8000B7B0011C1610011E17A0011136200119F
:10BDE800A97C00117B620011A97C0011AD620011D1
:10BDF800637C0011C1610011997A00113962001148
:10BE0800417C001100000000000000001F630011C9
:10BE1800417C00118163001145770011052A042A2D
:10BE2800012A002A022903280128002801180018DD
:10BE38000000000000000000000000000000008773
:10BE480001010201020101020102030304010301CD
:10BE5800010101010303020103000D000E0010009F
:10BE6800110013001401070108010A010B011C014C
:10BE78001D02040205020702080219021A021C0226
:10BE88001D0301030203170002010005040008074F
:10BE9800000B0A001716001D1C0102010105040110
:10BEA8000E0D011110011413011716011A190202BF
:10BEB80001020B0A020E0D021110021413021716CA
:10BEC800030504030807030B0A030E0D0001020310
:10BED80007090A0B0E0F101112141718191A1B1F35
:10BEE800202122005DA7001119A800110000000000
:10BEF8000200000036BE00110000000045B5001128
:0CBF0800000000000200000034BE001128
:020000041FFFDC
:1000000000000000153D001150BC00114CBC001157
:10001000B05BFF1F000000000000000000000000B7
:1000200000000000000000000000000000000000D0
:1000300000000000000000000000000000000000C0
:1000400000000000000000000000000000000000B0
:1000500000000000000000000000000000000000A0
:100060000000000000000000000000000000000090
:100070000000000000000000000000000000000080
:100080000000000000000000000000000000000070
:100090000000000000000000000000000000000060
:1000A0000000000000000000000000000000000050
:1000B0000000000000000000000000000000000040
:1000C0000000000000000000000000000000000030
:1000D0000000000000000000000000000000000020
:1000E0000000000000000000000000000000000010
:1000F0000000000000000000000000000000000000
:1001000000000000000000000000000000000000EF
:1001100000000000000000000000000000000000DF
:1001200000000000000000000000000000000000CF
:1001300000000000000000000000000000000000BF
:1001400000000000000000000000000000000000AF
:10015000000000000000000000000000000000009F
:10016000000000000000000000000000000000008F
:10017000000000000000000000000000000000007F
:10018000000000000000000000000000000000006F
:100190006D2DFF1FCD2BFF1FC16601000000000069
:1001A000000000000000000000000000000000004F
:1001B000000000000000000000000000000000003F
:1001C000000000000000000000000000000000002F
:1001D000000000000000000000000000000000001F
:1001E000000000000000000000000000000000000F
:1001F00000000000000000000000000000000000FF
:1002000000000000000000000000000000000000EE
:1002100000000000000000000000000000000000DE
:1002200000000000000000000000000000000000CE
:1002300000000000000000000000000000000000BE
:1002400000000000000000000000000000000000AE
:10025000000000000000000000000000000000009E
:10026000000000000000000000000000000000008E
:10027000000000000000000000000000000000007E
:10028000000000000000000000000000000000006E
:10029000000000000000000000000000000000005E
:1002A000000000000000000000000000000000004E
:1002B000000000000000000000000000000000003E
:1002C000000000000000000000000000000000002E
:1002D000000000000000000000000000000000001E
:1002E000000000000000000000000000000000000E
:1002F00000000000000000000000000000000000FE
:1003000000000000000000000000000000000000ED
:1003100000000000000000000000000000000000DD
:1003200000000000000000000000000000000000CD
:1003300000000000000000000000000000000000BD
:1003400000000000000000000000000000000000AD
:10035000000000000000000000000000000000009D
:10036000000000000000000000000000000000008D
:1003700091B5001100000000000000000000000026
:10038000000000000000000000000000000000006D
:10039000000000000000000000000000000000005D
:1003A000000000000000000000000000591AFF1FBC
:1003B000000000000000000000000000000000003D
:1003C000000000000000000000000000000000002D
:1003D000000000000000000000000000000000001D
:1003E000000000000000000000000000000000000D
:1003F00000000000000000000000000000000000FD
:081838009069FF1F4118FF1F1A
:10184000024981F3088801F0F7FF00009069FF1F4B
:1018500010B502F011F8072804D0122808D0022889
:1018600008D010BD044A0420136B01331363F8E75A
:101870000220F6E71420F4E76C5FFF1FF8B50700BD
:101880000C0026002500503630785135002804D150
:101890000300287058342370F8BD2978CA00481E08
:1018A0008141A3183800A25C5B68C9B2FFF7D0FF82
:1018B00000280DD12B78DA00A218013350602B706C
:1018C0003378044A013B3370136A01331362D8E75B
:1018D0000123DFE76C5FFF1F5C234343074910B51B
:1018E000C9180B0058331B78012B05D1FFF7C6FF31
:1018F000034A936A0133936210BDC046A05FFF1F85
:101900006C5FFF1F10B502F07FF8064A012113003B
:1019100010CB4942D967044B136001F06DFF2000E2
:1019200010BDC04600E100E01000100010B504003A
:1019300002F06AF8024B1C6001F05EFF10BDC04669
:1019400000E100E0431E5A425341A022F0B5D2010B
:101950005B421340154D164A40019B182A18127E0F
:101960008BB00191002A1BD01A000832D46F0022DC
:10197000E6B206AFE4B294420EDC2818C369002B2D
:1019800008D0019902AA117106AA049202AA16733C
:1019900003A898470BB0F0BD1978B9540132EAE7B3
:1019A0001A7D1A7806AB01261A70E6E72C62FF1F33
:1019B00000400040F0B5254B04004001C25C85B0FA
:1019C000002A2BD01A18117E002927D0917E0029D9
:1019D00024D01179022921D11689D788D168F51B25
:1019E000ADB22A1C102D00D9102292B2BE4217D1DE
:1019F0001818012303710023C269C38003819A422E
:101A000006D06846032103730171029301A8904731
:101A10000820002C00D0192001F08EF805B0F0BD90
:101A2000013C65426C41A0256442ED012C40084D0B
:101A30001B186419074D0633013A92B2AA42EDD041
:101A40001888461C1E80085C2070F5E72C62FF1F7A
:101A500000400040FFFF00000F220E4B10B59868B9
:101A6000104002380A280BD801F0F0FD0D0A0B0ACD
:101A70000A110A0A0A0A060002210020FFF762FF83
:101A800010BD0121F9E70020FFF794FFF8E7DB6FB5
:101A9000F6E7C046004000400F220E4B10B5986894
:101AA000104002380A280BD801F0D0FD0E0A0B0AAC
:101AB0000A120A0A0A0A060002210120FFF742FF61
:101AC00010BD01210800F9E70120FFF773FFF7E7D8
:101AD000DB6FF5E700900040564B70B51B68012B9B
:101AE00003D1554A936D0133936501F005FF534BC4
:101AF000534A1860534B544C1A600123534A1360E5
:101B0000534A13602378002B06D0062251495248CD
:101B100001F0A2FE00232370504A514B10681B783D
:101B2000C1B2002B0ED14F4CC0B223785BB2002B58
:101B30004FDB237824785BB264B21B0424021B19A8
:101B40001B1813600B1C50294ED95023464A474995
:101B50001078DBB2FF2202284BD10868444C454D77
:101B6000267890432A78964254D9227824782E7881
:101B7000023B5D10A31B6B435201D31A10335B1160
:101B80001843086001F028FF031F012B45D83A4B8A
:101B90001B78002B06D0394B1B78002B02D000207D
:101BA00001F02AFFA122364B92009978354B4A4327
:101BB0001B689B18832292009B181B78033B012B08
:101BC00003D8AF20400001F08FFD01222E4BDA82B6
:101BD00070BD237824785BB264B2FF33FF341B04FA
:101BE00024021B190138ABE7CAB2022AAED2022383
:101BF000ACE70868254C264D267890432A78964213
:101C000008D9227824782D78023B5B10641B63434B
:101C10005201B2E72378DBB2B2E70228D5D11D4BDF
:101C20001B78013B022B03D91B4B1B78022BCCD119
:101C30006C20C8E79809FF1FFC0FFF1FA45EFF1F61
:101C4000FF3F000014100340A85EFF1F0C1003406C
:101C500000100340D50BFF1F7211FF1FB40003409B
:101C60008C09FF1F680AFF1F490AFF1F94000340E9
:101C7000460AFF1F470AFF1FF908FF1F2209FF1F1F
:101C8000300DFF1F3409FF1FBC0BFF1F440AFF1F4D
:101C9000450AFF1F1C09FF1F2309FF1F10B501F094
:101CA0008BFE0022014B1A8010BDC046A25EFF1FB2
:101CB00070B5244D2B68002B28D001F04DFD2B680A
:101CC000D8402B680400002B27D001F0A5FE2B681C
:101CD000D8401D4B1D4A9978A1239B004B431268A5
:101CE000D118D25C91239B00002A20D0CA5801321F
:101CF000CA50174B17491B680868834214D3D23B5C
:101D0000181A012A1AD0144B186070BD01F024FD76
:101D1000124B196801F0C0FCD3E701F07DFE0F4BB8
:101D2000196801F0B9FCD4E70D495B18E8E7CA501F
:101D30000C4B1B68DB68E418201AE4E7F530FF3031
:101D4000E1E7C0461C08FF1F300DFF1F3409FF1FCD
:101D50009C09FF1FA45EFF1FA009FF1F1808FF1F9B
:101D60002DFF3F00AC5EFF1F70B504000D00282959
:101D700016D10300A433C2881B889B1A0B4A9BB25E
:101D800093420DD906006A3605223100653001F014
:101D900003FE002804D13100200001F025FE70BDB3
:101DA0002900200001F040FDF9E7C046FE7F000059
:101DB000F8B50500012001F0BFFD134CA36AA26A2B
:101DC0009342FBD1114E336001F076FC10490300C1
:101DD00008601048426894460F4A17680022BC45C4
:101DE00001D24268BA1A0D4802603268AD18A422C6
:101DF000E562606A520302436262094A1278002A6D
:101E000001D00F3B0B60F8BD00F00040340AFF1F0B
:101E1000E408FF1F28100040180AFF1F1C0AFF1FBC
:101E20001C09FF1F70B580241025E405A3682B430F
:101E3000A36001F049FCA368AB43A36070BD000040
:101E4000F7B5160080221C001023D205019191687D
:101E500005000B43936000225A4BD7301A6001F003
:101E60008BFC9D232A002F009B00EB58CA320121D6
:101E70000092FC37002B01D00021009A386801F055
:101E80000BFD2900009BCB311A784F4BD3351A60DC
:101E90004B780A781B0213438A7812041A43CB78D2
:101EA0001B061343494A1BBA13604B790A791B027C
:101EB00013438A7912041A43CB7931001B0613436A
:101EC000434A1BBA13606B782A781B021343AA7823
:101ED00012041A43EB781B0613433E4A1BBA1360E5
:101EE000019A330213433C4A13603C4B22001B1BF4
:101EF0009C4603293DDCB3089A0013005142B21AF4
:101F0000032A46D1354AE018511A827840781204E3
:101F100000020243E05C043302430A600022FF2B0C
:101F20004BDDF0222E4B12011A600F222D4B1A604E
:101F30002D4A1368002BFCD00023224A2749136046
:101F4000091B321D0B191B68043A180A23706070B4
:101F5000180C1B0EA070E3700434002AF2DC8022FF
:101F600010213B68D20501333B6093688B4393603B
:101F7000F7BD6346D578981893782D061B042B433C
:101F8000157804392B43557804322D022B43036016
:101F9000AFE7022A0AD1114AE05C511AE2185278DE
:101FA000120202430A6004339BB2B7E7012AB5D19B
:101FB0000A4A521AE15C1160F5E7084959180A60AB
:101FC0000433ACE7000004403C0004403800044007
:101FD00034000440300004400C0004400001044080
:101FE000040004401000044014000440F7B515003C
:101FF00080221C001023D2050091916807000B433A
:1020000093600023654AD730136001F0B5FB9D2330
:102010003E009B00F9583B00CA363200FC330029D1
:1020200000D07FE0586801F037FC390032785C4B13
:10203000CB311A604B780A781B0213438A78AC467E
:1020400012041A43CB78281D1B061343554A1BBAAA
:1020500013604B790A791B0213438A7912041A43DD
:10206000CB791B061343504A1BBA13604B7A0A7A8A
:102070001B0213438A7A12041A43CB7A21001B06EF
:1020800013434A4A1BBA1360009A2B021343484A6F
:1020900013602200474B1B1B0093009BCE785B18FC
:1020A00001938B7836061B0433430E780438334390
:1020B0004E78043136023343019E33600328ECDC52
:1020C0000321A808431C9B002940800003292BD131
:1020D0003849E5185E18A9786D78E35C09042D028B
:1020E000294319433160030008330021FF2B2DDD04
:1020F000314B324919600F21314B196001232749B7
:102100000B60304B19680029FCD006211B680B407E
:10211000042B20D080220020D20593680A318B4303
:102120009360FEBD01217DE7022908D121495D1898
:10213000E1184978E35C090219432960D3E70129D2
:10214000D3D11C495918E35C0B60CCE71948181827
:1021500001600433CAE7002310490B606346002B7B
:102160000CDC3B00FC335A68102101325A6080229B
:10217000D205936801208B439360D2E7009B9B18A4
:102180001B68190A13705170190C1B0ED3700423AD
:102190005B4291709C440432E0E7C046000004407A
:1021A0003C00044038000440340004403000044047
:1021B0000C0004400001044004000440080F00002B
:1021C000100004401400044010B5002901D001F0B3
:1021D000D3FB10BDF7B5604B01919978A1239B000B
:1021E0004B435E4A060014681022E418D6235B00B5
:1021F000E0583623FF33E35C00279343222B41D181
:10220000574B0F3A1A600760012501F0DDFB019B77
:102210001880E8235B00E35C002B01D0B34258DD5B
:102220000023504FFB70AD33FF33E3581A68002A88
:1022300003D09B88DB439B071DD03823FF33E35C2F
:10224000002B18D09B235B00E35C002B13D1D13310
:10225000FF33E35CB3420EDAA4235B00E15AE018DB
:10226000090A023101F0A0FB23000122FE33013EE6
:1022700001351A87FA70E8235B00E35C002B2AD053
:10228000A8B2FEBD03683D00002BBED0818804309B
:10229000090A023101F088FBD6235B00E3581F6076
:1022A000B2E72300B133BA00FF3398580137818871
:1022B0000430090A023101F077FBE8235B00E35C9C
:1022C000BB42EEDCE822F61AED1800235200A354BC
:1022D000A6E70027F1E7200001F036FA00281FD01A
:1022E000002E1DDD7319882647190193B6002000C2
:1022F00001F002FA5A3080002018406801358188C8
:102300000430090A023101F04FFB200001F0ACFA61
:10231000A3590133A351BD4202D0019B9D42E6D196
:10232000114BE35C002BABD095239B00E35C002BAF
:10233000A6D00E4BE15A0029A2D00D4AA35C9942C7
:1023400002D90133A3549BE700231A212000A35490
:1023500001F0B2FA94E7C046300DFF1F3409FF1FA9
:1023600000140340E010FF1F5A0200007202000038
:102370005E0200000D4970B54A6E0D4CD2038B69A8
:10238000D20BA24206D80B4D0224AA4204D901F076
:10239000EBF970BD02246442E21815007E2425404A
:1023A0002242F4D0A3432B438B61F0E700F00040BE
:1023B0000A200000FC1C00000B001B3B70B5040051
:1023C0003020E02B0DD81300E025493BFF3B9BB2AA
:1023D000ED00AB4205D8034B200019825A8201F070
:1023E000D3F970BD8410FF1FD722044B92009B5875
:1023F00010B5002B00D0984710BDC0460000FF1F4D
:1024000010B501F0ADF8FFF7EFFF2749274BCA6D74
:10241000274C1A4084235B001343CB65254B1B6874
:10242000186A01F089FA244B244A1A60244B254A81
:102430001A60A022244B52001A60244B187801F035
:1024400023FA2000224901F01FFB0023A36002337E
:10245000A360204B2049236003232048A36001F0A0
:1024600013FB10221E4BFF201A60802252031A60B9
:10247000802292031A60802212041A6001F0BCFAD2
:10248000012001F011FAFA20400001F02DFA582045
:1024900001F02AF9134801F017FA012001F044F97C
:1024A000072001F019FA10BD00F0004000FEFEFF09
:1024B00014100040AC5EFF1F000003400180063D89
:1024C000BC00034034080000A40003404A0AFF1F78
:1024D00071020000C3090000FFFF3F002810004008
:1024E00000E100E030750000674E336888331B68F8
:1024F00083F3088801F0C0F8644A65491368002036
:102500000B401360634B644A1B68934200D1A6E002
:1025100001F01AFA0221614A13688B431360FFF736
:102520006FFF5F4B5F4C1878C0B201F01DFA0023BB
:10253000A3600233A3605C4B0120236001F0FCF92F
:102540000323A36001F0E0F9040001F0D5F90500D0
:1025500001F0DAF9554B186001F06EFA544B196826
:10256000621A531EA14200D213008022D20393426A
:1025700001D39B029B0A3268D16AC90700D471E07B
:102580004C491C0C09689BB24C4359432402090A6C
:10259000641803264849FC3293680A6847489B1A26
:1025A000474A0768126847499B18474A9A183340B8
:1025B0009208DB190A600360042B03D9013233400F
:1025C0000A6003600E684149A619300001F064F802
:1025D0003F4F3E493B68C3183B603000019301F018
:1025E000E3F83C4E3068081838493060884205D915
:1025F000019B01333B6001F0D7F8316001F0DCF85A
:10260000354B1B78002B0DD001F076F9334B621B54
:10261000196812188A4232D24919091B091A30481E
:1026200001F032FA2F4E337A002B0ED001F064F90C
:10263000621BF1681218914224D94919091B091A21
:10264000294801F021FA00233372284B83F30888CC
:1026500001F062F8002001F077F901F02DFA01F0A5
:1026600073F95CE7DC0199000234641A5900641ABA
:1026700009214B438033CB40A408E41889E7FA21B1
:102680008900CCE71A49DBE7AC5EFF1F1CF0004075
:10269000FFFFC1FF0C0AFF1FB641210310000040DD
:1026A000490AFF1F14100040C3090000100AFF1F51
:1026B000340AFF1F380AFF1F200AFF1F280AFF1FC6
:1026C0001C0AFF1F240AFF1FC4090000710200003A
:1026D0006008FF1F2C0AFF1F1C09FF1FE408FF1FD3
:1026E00000100040740BFF1F3C1000400000002051
:1026F000DC050000A022054B92009B5810B5002B72
:1027000001D0984710BD01F017F8FBE70000FF1F4C
:10271000A122054B92009B5810B5002B01D0984781
:1027200010BD01F009F8FBE70000FF1FA222054BD6
:1027300092009B5810B5002B01D0984710BD00F0B7
:10274000FBFFFBE70000FF1FA322054B92009B58F5
:1027500010B5002B01D0984710BD00F0EDFFFBE74E
:102760000000FF1FA422054B92009B5810B5002BC0
:1027700001D0984710BD00F0DFFFFBE70000FF1F0E
:1027800070B501F0B9F84F4B186001F06DF9040015
:10279000C30702D401F040F870BD00224A4B1A6012
:1027A0004A4B18780138042829D800F04FFF03203D
:1027B000181C2400200001F037F90128ECD0444C0B
:1027C0002378042B6ED100F06FFF0028E4D001F0D5
:1027D00063F9582000F088FF02232370DCE7200013
:1027E00000F0DAFFE9E7200001F036F9E5E7200024
:1027F00001F00AF8E1E7200000F06EFFDDE701F0EC
:10280000EBF80500012808D1324B1B78053B012B62
:1028100003D82000FFF76EFFD1E72D4B1B78022B6A
:1028200001D0052B20D1022D28D12B4B9B7BAB4314
:102830001CD12000FFF76CFF264B18780128BED171
:102840006405BCD4244925224B7B034205D1233A9D
:1028500013405A42534126331A000B7D9342AED99E
:10286000322000F0C1FFAAE7022D07D1194B1B78D7
:10287000052B11D12000FFF759FFDDE7012D0BD10A
:10288000012B03D12000FFF75FFF98E7062B03D150
:102890002000FFF767FF92E7200000F04DFF022DB8
:1028A0008DD1C9E7032B04D10C4B987C00F08CFF31
:1028B00072E7072B00D06FE7094B987B00F0C4FF4D
:1028C0006AE7C0469C09FF1F9809FF1F9009FF1F78
:1028D0002309FF1F1C09FF1FA60BFF1FBC0BFF1FB7
:1028E000D40BFF1F10B500F099FE10BDF7B50B0C0F
:1028F000FF270122009300233C001E001D00944688
:10290000019089B262469A4010000840184136187A
:10291000B6B2FF2F02D1012E00D19FB20098024023
:102920001A41AD18ADB2FF2C02D1012D00D19CB2DD
:102930000133102BE6D10320012E07D1012D04D144
:10294000019B2401E4191C700138FEBD102EFCD13E
:102950000238102DF9D00230F7E700008023F7B5D8
:102960009C46264B264F01932649274A274D284C43
:10297000284B02281AD1604638600868264E30403D
:10298000802636033043086001990978002909D16F
:102990001660224A2A60224A2260E0221968914386
:1029A000A03A1BE08021C9021160F2E766463E6052
:1029B0000F68194E3E408027FF023E430E6001998A
:1029C000097800290DD1176001280ED1154A2A6017
:1029D000154A2260E02219689143C03A0A431A60FE
:1029E000F7BD802189021160EEE7E0210F4A024322
:1029F0002A600F4A22601A688A43F0E74B0AFF1FD9
:102A0000E0000340D8000340900003400000034072
:102A10005000034040000340FFFFE3FF0280063DFB
:102A2000804508220180063D8066082200800698C5
:102A300080550822F8B51E4B80261A680020140025
:102A40003440324232D11A681A4F32431A6001229E
:102A50003B68063093433B6000F06EFF0122164D49
:102A60002B681E432E603B680A2613433B60802779
:102A7000BF00124B1B683B4211D1013EF6B2FF2E44
:102A800009D17E220E4B1C682B68E40B1440934343
:102A900023432B6005E0082000F04EFFE9E7002EFD
:102AA000EFD180222B68600893432B60F8BDC046AD
:102AB000C4F000405CF0004018F0004068F00040B6
:102AC00060F0004010B500F01FFE01215820034ABD
:102AD00000F0DAFDFFF7AEFF10BDC046600AFF1F31
:102AE00010B578220021034800F076FE00F0C4FF04
:102AF000002010BDB461FF1F70B5040000F084FF1A
:102B000000230C200B4A010059438D18515C002909
:102B10000DD0A14208D1012300246B7000F034FFD6
:102B200000F06AFE200070BD01330A2BEBD11224A5
:102B3000F6E7C046B461FF1F70B5040000F064FF03
:102B4000002319001D000D4A1078002806D0A0426D
:102B50000CD1557001310C320A29F5D1002B0AD164
:102B600000F08AFF00F048FE002070BD5078461E3D
:102B7000B0411B18EEE700F007FFF3E7B461FF1F59
:102B8000F7B504000C20002384460E4D01926746E1
:102B90005F43E85D7E19A04212D000280BD10A4B9A
:102BA0009C4662461B7808331370019B70707C55FD
:102BB0007160B360FEBD01330A2BE8D10320F9E751
:102BC0000720F7E7B461FF1FB061FF1F8020F8B551
:102BD000484BC0051B68C1248360474BFF251A681A
:102BE000012313434361454BA4001A68444B402121
:102BF0001A60444B1A68444B1A60444B1A59AA4352
:102C00001A51C52292009E58AE43314380269950F6
:102C10009F583F49F6010F403E439E509E588027E3
:102C20003602360A3043985080201A5900020A4072
:102C300002431A5104341A59364E3F04324080265A
:102C40003A431A511A5936061202120A32431A51DD
:102C500008341A5980260A4002431A51C3229200AE
:102C60009F58B446AF4337439F509F58294E0F405B
:102C700007439F509F5837408026360437438026AD
:102C80009F509F5836063F023F0A37439F50C0224D
:102C90001F59AF433A431A511A591202120A1643E6
:102CA000C6221E5192009C58AC4365462C439C5052
:102CB0009C5800250C4020439850C72080001A588B
:102CC000154C1140C02212020A431A50134B1B78B4
:102CD000DB08AB4201DC0020F8BD2378002B06D0D6
:102CE000A368002B00D0984701350C34EEE7122082
:102CF000F2E7C046DC3DFF1FD83DFF1FB0F00040AB
:102D0000AC61FF1FB4F00040A861FF1F00E100E0CC
:102D1000FF00FFFFFFFF00FFB461FF1FB061FF1F57
:102D2000030010B51F2809D80722002013400724EC
:102D300004490A78A24313430B7010BD00230620F8
:102D4000F5E7C046B061FF1F054B06491B780A68CE
:102D500005485B0702401B0B134300200B607047C4
:102D6000B061FF1F1CF00040FFFFC1FF70B50C25D4
:102D7000FFF7EAFF0A4B1C780A4BE4086543ED189D
:102D8000002C01D1200070BD2B78002B06D06B6881
:102D9000002B00D09847013C0C3DF1E71220F2E7F0
:102DA000B061FF1FA861FF1F1FB5002102220B00A9
:102DB00001910091052000F077FE02230B490A687B
:102DC0001A42FCD120230393039B5A1E0392002B2B
:102DD000FAD1074A1368002BFCDA0B246C4420005C
:102DE000012100F0A1FD207804B010BD90C8004082
:102DF00000C8004013B504000A4B0193019B002B4F
:102E000001D1112016BDFFF7CFFF2300034004427C
:102E100005D0052000F090FD019B013BEDE7180077
:102E2000F0E7C046FFFFFF0707B500F0EDFD802289
:102E30000821D205936A0191002B01D107399162D3
:102E400002210C4A11600199481E01900029FAD113
:102E500003311160053101910199481E019000294B
:102E6000FAD11160002B02D18022D205936200F0CA
:102E7000C3FC07BD00C00040F0B52D4C89B02378DD
:102E8000002B4FD1FEF73EFD02232A4F03903A68F4
:102E90001A42FCD120230693069B5A1E0692002B51
:102EA000FAD1254E3368002BFCDA0120FFF7A2FF90
:102EB000011E02D0112009B0F0BD030003220190D1
:102EC000009005AD9F2000F0EFFD0321280000F0E9
:102ED0002BFD02233A681A42FCD120230793079B5B
:102EE0005A1E0792002BFAD13368002BFCDA01201E
:102EF000FFF780FF0028DDD10398FEF717FDAA78C1
:102F00006B7811041B020B4329780B436360130099
:102F1000113B0A49052B07D801239340A3600B609E
:102F2000012323700020C6E780231B03F6E7C04679
:102F3000C43DFF1F90C8004000C800409808FF1F14
:102F40001E4B30B55A6818781D4B85B0D3185942BE
:102F50004B4101210093002300F076FD194B1A4AE2
:102F600002259A6300221A6510325A658022C42114
:102F70009D65164B1648D202DA6789004258154BF8
:102F800080241A4080231B041343435064234120B0
:102F90000393E40500F006FA402000F003FA6562AE
:102FA000039D6B1E0393002DFAD103236362FFF789
:102FB0003BFFA562FFF760FF05B030BDD03DFF1FAE
:102FC00095FFFEF700C80040050001FF04E100E0A6
:102FD00000E100E0FFFF00FFF0B585B00700FEF75D
:102FE00091FC022305002D4C22681A42FCD12023BB
:102FF0000093009B5A1E0092002BFAD1284E336892
:10300000002BFCDA0120FFF7F5FE002803D0112485
:10301000200005B0F0BD234B2360022322681A4232
:10302000FCD120230193019B5A1E0192002BFAD15F
:103030003368002BFCDA0120FFF7DCFE0028E6D124
:10304000194B1F60022322681A42FCD120230293ED
:10305000029B5A1E0292002BFAD13368002BFCDA35
:103060000120FFF7C7FE0028D1D1104B23600223B7
:1030700022681A42FCD120230393039B5A1E039219
:10308000002BFAD13368002BFCDA0120FFF7B2FEE7
:10309000041EBCD12800FEF749FCB9E790C80040E7
:1030A00000C8004001000006A8C8004001800001DF
:1030B00010B50020FFF790FF10BD000010B5064BC3
:1030C00018705960FFF73CFF00211320034AFFF7F7
:1030D00057FD002010BDC046D03DFF1F412FFF1FF0
:1030E000F0B5040085B003920291FEF70BFC882234
:1030F00063035B0B52051A438023DB059D6A802323
:10310000274F0092BA68002601901B039A420CD9FF
:10311000F82326001B041E401C4206D08022214BAF
:1031200052025E6219680A431A60002D0BD100F04A
:103130006BFC02221C4B1A608023DB055A62013AA9
:103140009A6200F059FB0023039A934220D1002D8C
:103150000AD100F059FC144B03221D608023DB05CB
:103160005A629D6200F048FB8023BA681B039A42B2
:1031700008D9002E06D000220A4B0C495A621A6860
:103180000A401A600198FEF7D1FB002005B0F0BD9F
:10319000009A0299D2181278CA540133D4E7C04673
:1031A000C43DFF1F00C8004000C00040FFFFFEFFFD
:1031B000F0B587B0029103920400FEF7A3FB0190E3
:1031C00000F022FC802302250122234EDB0535601E
:1031D0005D629A6200F010FB204F3B682B42FCD1ED
:1031E00020230493049B5A1E0492002BFAD11C4DF9
:1031F0002B68002BFCDA0120FFF7FCFD002802D031
:10320000112007B0F0BD2000039A029900F0A4FB42
:10321000022304003A681A42FCD120230593059B3F
:103220005A1E0592002BFAD12B68002BFCDA0120E4
:10323000FFF7E0FD051EE3D100F0E6FB802303224B
:10324000DB0535605A629D6200F0D6FA0198FEF700
:103250006DFBE0B2D5E7C04600C0004090C800401A
:1032600000C80040F0B5802489B00600FEF74AFB94
:10327000E405A36A02250393029000F0C5FB012335
:10328000304F3D606562A36200F0B6FA2E4C2368B1
:103290002B42FCD120230593059B5A1E0592002B3F
:1032A000FAD12A4D2B68002BFCDA0120FFF7A2FD92
:1032B000002803D01124200009B0F0BD244B236066
:1032C000022322681A42FCD120230693069B5A1E31
:1032D0000692002BFAD12B68002BFCDA0120FFF7B5
:1032E00089FD021EE6D11B4B03211E6003000190E5
:1032F0000090202000F0D8FB022322681A42FCD163
:1033000020230793079B5A1E0792002BFAD12B68A4
:10331000002BFCDA0320FFF76DFD041ECAD100F07C
:1033200073FB80230322DB053C605A629C6200F041
:1033300063FA039B002B01D1FFF776FD0298FEF79D
:10334000F5FAB8E700C0004090C8004000C800404F
:103350000100000694C8004007B500020191042254
:10336000000A01A9FFF724FF0EBD000073B5050098
:1033700005240B4AA3005B429B1819686B46DE1DAF
:103380003000FFF7B3FA022804D133782B55013C03
:10339000EFD276BD052CFCD00128FAD10230F8E737
:1033A000140900111F2807D8012380228340D20569
:1033B00091680B43936070473F2808D8012380220F
:1033C00020388340D20551690B435361F3E75F28EE
:1033D000F1D80123802240388340D205116A0B4383
:1033E0001362E8E71F2807D8012280218240C9051F
:1033F0008B6893438B6070473F2808D80122802157
:1034000020388240C9054B6993434B61F3E75F283D
:10341000F1D80122802140388240C9050B6A9343CC
:103420000B62E8E71F2810D880230200DB05153A5D
:103430001968012A06D820229143196019680A43A5
:103440001A60704701228240F6E73F2811D8802396
:103450000200DB05353AD968032A06D810229143C9
:10346000D960D9680A43DA60EBE70122203882404C
:10347000F5E75F28E5D842238022181A413B8340B4
:10348000D205516A99435162516A0B435362D8E79E
:1034900010B50400012813D1A022184992050B6829
:1034A0005B015B0913430B60154B164A1968114009
:1034B000154A0A431A60402219680A431A6010BD6F
:1034C0000028FCD101000A2000F0FEFA21000B20A8
:1034D00000F0FAFAC0220A4B920019680A43402110
:1034E0001A601A688A431A60B022044912060B68EF
:1034F0005B015B0913430B60E1E7C04614F0004039
:103500001CF000407F00FEFF80FD010072B6074AFC
:103510001368013313600422054B1A600023054A27
:1035200013608022D2055360FEE7C0467808FF1F73
:10353000C0F00040C4F0004005490B68002B05D1E5
:10354000044A0A6004490A60044A13607047C0468E
:10355000140AFF1F841E0000380AFF1FC4F0004039
:103560000023034A1360034A1360034A1360704741
:1035700054F0004040F1004044F10040002310B5F9
:10358000184C8AB0009301932378012B27D0694609
:10359000012000F0C1F9002817D1009B12490293C5
:1035A000019B06AA0393114B02A81B680493104BBE
:1035B0001B68059300F088F810220E4906A800F059
:1035C000EBF9002804D1FF23237000200AB010BDBE
:1035D0000123094A074902A8237000F075F8012069
:1035E000F4E7C046B05EFF1F102900110829001142
:1035F0000C29001120290011B45EFF1F13B501240E
:103600006946012000F088F9034B00940193FFF70D
:10361000B5FF200016BDC046BB0B000010B5FFF77C
:103620009FFFFFF7EBFF002802D0024B984710BD29
:10363000FEE7C046E1A2000002B471464908490015
:10364000095649008E4402BC7047C04602B4714618
:1036500049084900095C49008E4402BC7047C046D5
:1036600003B47146490840004900095A49008E4494
:1036700003BC70470000000001B40248844601BC4E
:10368000604700BFC9A9000001B40248844601BCDC
:10369000604700BF0167010001B40248844601BCD5
:1036A000604700BF090E000001B40248844601BC17
:1036B000604700BF01D7000001B40248844601BC46
:1036C000604700BFBD5C010001B40248844601BCF4
:1036D000604700BFDD3F000001B40248844601BCE2
:1036E000604700BFF935010001B40248844601BCBF
:1036F000604700BF7912010001B40248844601BC52
:10370000604700BFD9B0000001B40248844601BC44
:10371000604700BFED68010001B40248844601BC67
:10372000604700BF7997000001B40248844601BC9D
:10373000604700BFE512010001B40248844601BCA5
:10374000604700BFE917010001B40248844601BC8C
:10375000604700BF71B0000001B40248844601BC5C
:10376000604700BFE90B010001B40248844601BC78
:10377000604700BFD1AE000001B40248844601BCDE
:10378000604700BF8944000001B40248844601BC80
:10379000604700BF116E000001B40248844601BCBE
:1037A000604700BF0934010001B40248844601BCEF
:1037B000604700BF090E000001B40248844601BC06
:1037C000604700BFD544010001B40248844601BCF3
:1037D000604700BF4DF9000001B40248844601BCB7
:1037E000604700BFB70E000001B40248844601BC28
:1037F000604700BF6137010001B40248844601BC44
:10380000604700BF9DA9000001B40248844601BC86
:10381000604700BFF535010001B40248844601BC91
:10382000604700BFDD0A010001B40248844601BCC4
:10383000604700BF51B8000001B40248844601BC93
:10384000604700BF99B5001101B40248844601BC2D
:10385000604700BFC1F7000001B40248844601BCC4
:10386000604700BFE94C010001B40248844601BC36
:10387000604700BF5976010001B40248844601BC8C
:10388000604700BFE927000001B40248844601BC3C
:10389000604700BFEDA5000001B40248844601BCAA
:1038A000604700BF2144000001B40248844601BCC7
:1038B000604700BF6911010001B40248844601BCA1
:1038C000604700BF53B9000001B40248844601BC00
:1038D000604700BF8D11010001B40248844601BC5D
:1038E000604700BFF90D010001B40248844601BCE5
:1038F000604700BF8512010001B40248844601BC44
:10390000604700BFC95C010001B40248844601BCA5
:10391000604700BF156B010001B40248844601BC3A
:10392000604700BFE1AC000001B40248844601BC1E
:10393000604700BF3D71010001B40248844601BCEC
:10394000604700BF0189000001B40248844601BC01
:10395000604700BF016C010001B40248844601BC0D
:10396000604700BF9573010001B40248844601BC62
:10397000604700BF8914010001B40248844601BCBD
:10398000604700BFE9D4000001B40248844601BC8E
:10399000604700BF21A9000001B40248844601BC71
:1039A000604700BFCD4C010001B40248844601BC11
:1039B000604700BFC115010001B40248844601BC44
:1039C000604700BF8D82000001B40248844601BCFC
:1039D000604700BFCD0C010001B40248844601BC21
:1039E000604700BFDD0C010001B40248844601BC01
:1039F000604700BF85C1000001B40248844601BC95
:103A0000604700BFED6B010001B40248844601BC71
:103A1000604700BF75A9000001B40248844601BC9C
:103A2000604700BF6D0B010001B40248844601BC31
:103A3000604700BF0134010001B40248844601BC64
:103A4000604700BFC166010001B40248844601BC62
:103A5000604700BFC56D010001B40248844601BC47
:103A6000604700BF0534010001B40248844601BC30
:103A7000604700BFBD0B010001B40248844601BC91
:103A8000604700BFADAE000001B40248844601BCEF
:103A9000604700BF2D6C010001B40248844601BCA0
:103AA000604700BF6DF6000001B40248844601BCC7
:103AB000604700BF496D010001B40248844601BC63
:103AC000604700BF8552010001B40248844601BC32
:083AD000604700BF1DA20011B8
:103AD8000200000032BE00110100000040BC0011CD
:103AE800020000002EBE001101000000183BFF1F5D
:103AF8000200000048BC001101000000305CFF1FFC
:103B0800020000002CBE001103000000A45BFF1F90
:103B1800120000000200000032BE00110100000087
:103B280088BC0011020000002EBE00110100000038
:103B380085BC00110200000092BC001103000000C7
:103B4800DF5BFF1F020000002CBE00110300000015
:103B5800F45BFF1F020000002EBE001101000000F0
:103B680084BC00110200000090BC0011030000009A
:103B7800B55BFF1F020000002CBE0011030000000F
:103B8800D65BFF1F0200000032BE001101000000DA
:103B9800CCBC0011020000002EBE00110100000084
:103BA800613CFF1F02000000DEBC001101000000A4
:103BB800C3BC0011020000002EBE0011010000006D
:103BC800603CFF1F02000000DCBC00110100000087
:103BD800FC5BFF1F020000002EBE00110100000068
:103BE8005F3CFF1F02000000DABC0011010000006A
:103BF800B3BC0011020000002EBE0011010000003D
:103C08005E3CFF1F02000000D8BC0011010000004C
:103C1800AEBC0011020000002EBE00110100000021
:103C28005D3CFF1F02000000D6BC0011010000002F
:103C3800A9BC0011020000002EBE00110100000006
:103C48005C3CFF1F02000000D4BC00110100000012
:103C5800A4BC0011020202020202000000000000DF
:103C680016150000954B00115B4B001120BD00118B
:103C780090011D0018001800FFFF0701020304054A
:103C8800060201060000000000000000000000001D
:103C9800000000000000000000000000000000001C
:103CA800030000000200000032BE00110100000005
:103CB80040BD0011020000002EBE001101000000EE
:103CC8001C3DFF1F020000004ABD0011010000005A
:103CD8002A5CFF1F020000002CBE00110300000038
:103CE800945EFF1F020000002EBE001101000000BC
:103CF8001C3DFF1F0200000048BD0011010000002C
:103D08002C5CFF1F020000002CBE00110300000005
:103D18008C5EFF1F120800000000000000C6C600ED
:103D28000000000000000000131100000001000066
:103D380000000111FFFF0000504859360000000044
:103D4800000000000B000500F0000000B40000288F
:103D5800002800283075A000A000A000A0000008DE
:103D68000008E001F0001000100010001000100022
:103D7800100050005000500010001000D007000044
:103D8800000000000F00010005003075070010005A
:103D9800010081FF00000000FF0000000574001111
:103DA8000D7200119D6F0011FFFF0100FF00000060
:103DB800219E00119D9B0011B59A00110000000082
:103DC8000000000000000800040000003B0001089B
:103DD8005902E001882128000200000032BE0011CB
:103DE80001000000F8BE0011020000002EBE001104
:103DF800010000005D3EFF1F020000002ABE001106
:103E0800010000006C62FF1F020000002EBE0011BE
:103E1800010000005C3EFF1F0200000028BE0011E8
:103E2800010000005A3EFF1F020000002EBE0011D4
:103E380001000000583EFF1F0200000026BE0011CE
:103E480001000000503EFF1F180018001D009001DF
:103E580002000003020200000200000032BE00114E
:103E6800010000000CBF0011020000002EBE00116E
:103E780001000000A03EFF1F0200000024BE001148
:103E88000000000000000000020000002CBE00112D
:0A3E9800030000008C62FF1F20FFF2
:040000051FFF184180
:00000001FF
